:1019100020002A2A2000202A2A0020204164647204
:101920006573733A202020253034580020205265FA
:10193000766973696F6E3A202025730050483A2506
:10194000352E3266620050493A25352E31670048FF
:10195000653A25352E316625250054483A25352E21
:101960003166254B0046563A25352E316625250031
:1019700042563A25352E31662525004C4E324D30E3
:10198000004C4E324D3120004C4E324131004C4E15
:10199000324130004854524D30004854524D3120AD
:1019A000004854524131004854524130002B2048E5
:1019B00045412D002B204845202D00425453002442
:1019C00049643A207363735F313030315F627473FE
:1019D0002E63203330383320323030362D30342DE2
:1019E00032362031343A31393A34385A20726974F7
:1019F0007420240001340000004572726F720000F0
:101A00000001000D000000000000000000000000C8
:101A10000000000134000000537461746500000090
:101A200001000E00000000411000003F8000000097
:101A3000000001340000004C4E32565300000001FB
:101A4000000F00000000400000003F800000000088
:101A5000000134000000485452530000000001000F
:101A60001000000000400000003F80000000000067
:101A700002030000004C4E32206F6E000001001186
:101A80000000000042F000004120000000000002C1
:101A9000030000004C4E32206F6666000100130008
:101AA000000000456100004120000000000002032A
:101AB0000000005072656865617400010015000047
:101AC0000000427000003F80000000000001340070
:101AD00000004B41204F757400000100170000000A
:101AE0000040E000003F80000000000001340000E2
:101AF000004B4120496E000000010018000000006A
:101B00000000000000000000000000045A00000176
:101B10004B41204C6576656C010019000000000007
:101B20000000000000000000000001320000004C36
:101B30004E3220766C766501001D000000003F806B
:101B400000003F80000000000001320000004C4E09
:101B500032206874720001001E000000003F800007
:101B6000003F80000000000004070000014C4E32DE
:101B7000766C76205401001F000000000000000079
:101B80000000000000000004070000014C4E326815
:101B900074722054010023000000000000000000C7
:101BA000000000000000045A0000014A542046765C
:101BB0006C76650100270000000042C800003F80ED
:101BC0000000000000045A0000014A542042766CD4
:101BD000766501002B0000000042C800003F800035
:101BE0000000000004070000014A542054000000D7
:101BF0000001002F000000000000000000000000B5
:101C0000000000045A0000014C4865206C766C31DD
:101C10000100330000000000000000000000000090
:101C20000000045A0000014C4865206C766C3201BB
:101C3000003700000000000000000000000000006D
:101C40000004070000014C4E3220546C00000100DB
:101C50003B00000000000000000000000000000049
:101C600004070000014C4E32205472000001003F76
:101C70000000000000000000000000000000000460
:101C8000070000014C4E3220547700000100430051
:101C90000000000000000000000000000000040739
:101CA0000000014C4E322054740000010047000037
:101CB0000000000000000000000000000004070019
:101CC00000014C4845205444630001004B000000D3
:101CD00000000000000000000000000004070000F9
:101CE000014C48452054446C0001004F00000000A6
:101CF00000000000000000000000000407000001D8
:101D00004C4845205444720001005300000000007C
:101D10000000000000000000000004070000014C6B
:101D200048452054526300010057000000000000A5
:101D300000000000000000000004070000014C4803
:101D4000452054526C0001005B00000000000000C0
:101D5000000000000000000004070000014C48459E
:101D6000205452720001005F0000000000000000DB
:101D7000000000000000000416FD00014C4E32205F
:101D8000500000000100630000000000000000009F
:101D900000000000000004160000014C48452050DF
:101DA00000000001006700000000000000000000CB
:101DB000000000000004180000015175656E6368A2
:101DC000310001006B000000000000000000000076
:101DD0000000000004180000015175656E63683250
:101DE0000001006F00000000000000000000000083
:101DF000000000045A0000014C484520446D640076
:101E0000010073000000000000000000000000005E
:101E100000000418000009414443300000000001A4
:101E2000007700000000000000000000000000003B
:101E30000004180000094144433100000000010083
:101E40007B00000000000000000000000000000017
:101E50000418000009414443320000000001007FE3
:101E6000000000000000000000000000000000046E
:101E700018000009414443330000000001008300C2
:101E80000000000000000000000000000000041836
:101E900000000941444334000000000100870000B5
:101EA0000000000000000000000000000004180016
:101EB0000009414443350000000001008B00000090
:101EC00000000000000000000000000004180000F6
:101ED00009414443360000000001008F000000006B
:101EE00000000000000000000000000418000009CD
:101EF000414443370000000001009300000000004F
:101F0000000000000000000000000418000009416B
:101F10004F465330000000010097BDCCCCCD3DCCE6
:101F2000CCCD3A83126F0000000418000009414F25
:101F300046533100000001009BBDCCCCCD3DCCCC44
:101F4000CD3A83126F0000000418000009414F468B
:101F5000533200000001009FBDCCCCCD3DCCCCCD98
:101F60003A83126F0000000418000009414F4653E5
:101F7000330000000100A3BDCCCCCD3DCCCCCD3A8C
:101F800083126F0000000418000009414F465334CB
:101F90000000000100A7BDCCCCCD3DCCCCCD3A8318
:101FA000126F0000000418000009414F465335002D
:101FB00000000100ABBDCCCCCD3DCCCCCD3A8312E2
:101FC0006F0000000418000009414F46533600001E
:101FD000000100AFBDCCCCCD3DCCCCCD3A83126F4F
:101FE0000000000418000009414F4653370000006C
:101FF0000100B3BDCCCCCD3DCCCCCD3A83126F002B
:102000000000045D000009414741494E30000001D5
:1020100000B73F6666663F8CCCCD3A83126F0000F6
:1020200000045D000009414741494E3100000100B4
:10203000BB3F6666663F8CCCCD3A83126F000000D2
:10204000045D000009414741494E3200000100BFD4
:102050003F6666663F8CCCCD3A83126F0000000469
:102060005D000009414741494E3300000100C33F74
:102070006666663F8CCCCD3A83126F000000045D2B
:10208000000009414741494E3400000100C73F6646
:1020900066663F8CCCCD3A83126F000000045D0071
:1020A0000009414741494E3500000100CB3F6666BB
:1020B000663F8CCCCD3A83126F000000045D0000B7
:1020C00009414741494E3600000100CF3F66666630
:1020D0003F8CCCCD3A83126F000000045D000009F4
:1020E000414741494E3700000100D33F6666663FD5
:1020F0008CCCCD3A83126F0000000418000019390F
:1021000031305F303000000100D7000000000000D7
:10211000000000000000000100041800001939311F
:10212000305F303100000100DB00000000000000E3
:1021300000000000000001010418000019393130CE
:102140005F303200000100DF0000000000000000EE
:102150000000000000010204180000193931305F4E
:10216000303300000100E300000000000000000028
:1021700000000000010304180000193931305F30FD
:102180003400000100E70000000000000000000033
:10219000000000010404180000193931305F3035A7
:1021A00000000100EB000000000000000000000043
:1021B0000000010504180000193931305F30360085
:1021C000000100EF0000000000000000000000001F
:1021D00000010604180000193931305F3037000063
:1021E0000100F300000000000000000000000000FB
:1021F000010704180000193931305F303800000140
:1022000000F70000000000000000000000000001D6
:102210000804180000193931305F3039000001001E
:10222000FB000000000000000000000000000109A9
:1022300004180000193931305F313000000100FF0F
:1022400000000000000000000000000000010A047F
:10225000180000193931305F3131000001010300ED
:10226000000000000000000000000000010B041846
:102270000000193931305F313200000101070000E0
:102280000000000000000000000000010C04180025
:1022900000193931305F3133000001010B000000BB
:1022A00000000000000000000000010D0418000004
:1022B000193931305F3134000001010F0000000096
:1022C000000000000000000000010E0418000019CA
:1022D0003931305F3135000001011300000000008A
:1022E0000000000000000000010F04180000193970
:1022F00031305F313600000101170000000000009E
:10230000000000000000000110041800001939311D
:10231000305F3137000001011B00000000000000A9
:1023200000000000000001110418000019393130CC
:102330005F3138000001011F0000000000000000B4
:102340000000000000011204180000193931305F4C
:1023500031390000010123000000000000000000EE
:102360000000000001130000000000000000000059
:10237000000000000000000000000000000000005D
:05238000000000000058
:10606B0001A1010376FF19F4C113C114C115C116A7
:10607B004400000000000044000900000000410043
:02608B0008000B
:104D3F00E4F584F5BA75BCE075E880F5D1F58475B6
:104D4F00D102F58475D48075840175D48075840F74
:104D5F0075A4F575A5BF75A6FF75A7FFEF6059E49C
:104D6F00F53F75F004E53FA42497F582E5F0340094
:104D7F00F5831216770000000075F004E53FA424B8
:104D8F00B7F582E5F03400F5831216773F80000007
:104D9F00053FE53FB408CB900011E4F0A3743CF05D
:104DAF00A3E4F0A374FAF0A3E4F0A3740AF0900064
:104DBF007312167742700000E4F584E5EF20E113DB
:104DCF00780D7C007D017B017A0179277E017F1AA6
:104DDF001213E4E490000DF0F53FAF3F12476C055E
:104DEF003FE53FC3946340F27D087F01126397E470
:104DFF00FDFF126754E4F53F7B007A00790F120034
:104E0F000E7C007D02121496C374079FFFE49EFE72
:104E1F00C3E53F9FEE6480F8748098500D7BFF7A56
:104E2F00197910126604053F80CE7BFF7A1979122B
:104E3F001266047B007A00790F1266047BFF7A19E1
:104E4F0079161266047D01E4FF1267547BFF7A190D
:104E5F00791A850949850A4A123E9F7D02E4FF129D
:104E6F00675478117C037D017BFF7A1979D3121770
:104E7F00EB7B017A0379117D20126720E412145025
:104E8F00754901754A03754B117BFF7A19792C12FD
:104E9F003E9FE490000DF0A3E0D394034002E4F0B2
:104EAF0090000FE0D394024002E4F0900010E0D3A2
:064EBF0094024002E4F041
:014EC50022CA
:0C476C00157CA87CEFF6E57C24FAF57CB7
:104778002406F8E624F9603A24FD606F1460782472
:10478800FD700302480B1470030248C1240D600336
:1047980002497490000FE0FF700690001DF0800A37
:1047A800EFB4010690001D7401F07F0A12476C02F5
:1047B8004974900017E0FF20E003D38001C392B44E
:1047C800EF20E103D38001C392B5900017E0FF20EA
:1047D800E203D38001C392B6900131E06F70030207
:1047E8004974D21B788976F102497490001DE0243F
:1047F800FFB392B002497490001EE024FFB392B751
:10480800024974E4FFFE7D807C41900027E0F8A314
:10481800E0F9A3E0FAA3E0FB120E28E4FBFA79C85A
:104828007842120F31E4FBFA79807840120D37A8EC
:104838007C12165FA87CE8C0E01216037BAE7A47AC
:104848007961783E120D33D0E0F812165FE4FBFA76
:1048580079C07841E8C0E0A87C121603D0E0F812CD
:104868000F31E4FBFA79807845120E28121079E5A9
:104878007C2404F8EEF608EFF6E57C2404F9C3E797
:104888009410400AE57C2404F8760F0876FFE57C4E
:104898002404F9C3E794005009E57C2404F8E4F6FD
:1048A80008F6E4F584E57C2404F808E6F5D2E57C0E
:1048B8002404F9E7F5D3024974E4FFFE7D807C41C6
:1048C80090002BE0F8A3E0F9A3E0FAA3E0FB120EB6
:1048D80028E4FBFA79C87842120F31E4FBFA7980B0
:1048E8007840120D37A87C12165FA87CE8C0E01249
:1048F80016037B0A7AD779A3783E120D33D0E0F8F5
:1049080012165FE4FBFA79C07841E8C0E0A87C128F
:104918001603D0E0F8120F31E4FBFA7980784512DB
:104928000E28121079E57C2404F8EEF608EFF6E577
:104938007C2404F9C3E79410400AE57C2404F87643
:104948000F0876FFE57C2404F9C3E794005009E5D5
:104958007C2404F8E4F608F6758401E57C2404F860
:0C49680008E6F5D2E57C2404F9E7F5D35D
:07497400E57C2407F57C221D
:0567C4008F357F00226B
:10657F008B358A36893712140AAB38AA39A93A12E1
:10658F001450AB35AA36A937900001121423AB383B
:0D659F00AA39A93A9000011214627F02226D
:10673C007B01900315E0FCA3E0FDA3E0FEA3E0FFCA
:08674C00C2AF1215E9D2AF2221
:085D2D008B408A4189428D433D
:105D3500E4900325F0A31216773F80000090032519
:105D4500E0C395435024A3E0FCA3E0FDA3E0FEA33C
:105D5500E0FFE4FBFA79207841120E289003261221
:105D6500166B900325E004F080D3AB40AA41A9420D
:105D7500121599900326E0F8A3E0F9A3E0FAA3E051
:105D8500FB120E28E4FBFAF9783F120D371257DDA6
:105D9500900326E0F8A3E0F9A3E0FAA3E0FB120FD5
:0A5DA50031AB40AA41A9420215E902
:0A4B72008E3B8F3C8B3D8A3E893F4D
:104B7C00E4F584E53C540FF5BB75BCE090031F7461
:104B8C0004F0A3E4F090031912167700000000E47F
:104B9C0090031DF0A3F090031FE0FEA3E0FFC39071
:104BAC00031EE09F90031DE09E504CC2AFE4F584C1
:104BBC00C2EDD2EC30EDFDD2AF900319E0F8A3E0DA
:104BCC00F9A3E0FAA3E0FBAFBFEFFEADBEEDFFE44F
:104BDC00FCFDEB2FFFEA3EFEED39FDEC38FC9003BB
:104BEC001912166B12002690031EE004F070A790A9
:104BFC00031DE004F0809F900319E0FCA3E0FDA3EB
:104C0C00E0FEA3E0FF780612158690031912166BCE
:104C1C00C3E53C9402E53B64809480900319E0FC6E
:104C2C00A3E0FDA3E0FEA3E0FFE4502312103BE45D
:104C3C00FBFA79807847120F31E4FBFA79A07841BE
:104C4C00120E28E4FBFA792078C1120D3780171266
:104C5C00103BE4FBFA79807847120F31E4FBFA79C8
:104C6C00207841120E2890032112166B900321E03C
:104C7C00FCA3E0FDA3E0FEA3E0FFECC0E0EDC0E090
:104C8C00EEC0E0EFC0E0E53CAE3B7802C333CE3380
:104C9C00CED8F92497F58274003EF583E0F8A3E0B2
:104CAC00F9A3E0FAA3E0FBD0E0FFD0E0FED0E0FDFA
:104CBC00D0E0FC120D3390032112166B900321E00F
:104CCC00FCA3E0FDA3E0FEA3E0FFECC0E0EDC0E040
:104CDC00EEC0E0EFC0E0E53CAE3B7802C333CE3330
:104CEC00CED8F924B7F58274003EF583E0F8A3E042
:104CFC00F9A3E0FAA3E0FBD0E0FFD0E0FED0E0FDAA
:104D0C00D0E0FC120E2890032112166B7B017A0363
:104D1C0079217D03125D2DC2AF900321E0FCA3E04D
:104D2C00FDA3E0FEA3E0FFAB3DAA3EA93F1215E9AF
:024D3C00D2AFF4
:014D3E002252
:1055A800C297D296D2957F017E00125FADC295E474
:1055B800F53E309603433E04D2977F017E00125F8A
:1055C800ADC2977F017E00125FAD309603433E085F
:1055D800D2977F017E00125FADC2977F017E0012D5
:1055E8005FAD309603433E01D2977F017E00125F84
:1055F800ADC2977F017E00125FAD309603433E0235
:10560800D2977F017E00125FADC2977F017E0012A4
:105618005FADE53EF45407900018F0A296921AD2B6
:10562800977F017E00125FADC2977F017E00125FF7
:10563800ADA2969219D2977F017E00125FADC297F4
:105648007F017E00125FADA2969218D2977F017EED
:1056580000125FADC2977F017E00125FADA29692E5
:01566800172A
:01566900221E
:1038DE003008031267B1E4FDFF1267547BFF7A19BB
:1038EE00793C900067E0FCA3E0FDA3E0FEA3E0F5C9
:1038FE004C8E4B8D4A8C49123E9FE4FD7F0A126717
:10390E00547BFF7A197946900063E0FCA3E0FDA397
:10391E00E0FEA3E0F54C8E4B8D4A8C49123E9F7D06
:10392E0001E4FF1267547BFF7A19794F900033E060
:10393E00FCA3E0FDA3E0FEA3E0F54C8E4B8D4A8C7C
:10394E0049123E9F7D017F0A1267547BFF7A1979D7
:10395E005A900057E0FCA3E0FDA3E0FEA3E0F54C77
:10396E008E4B8D4A8C49123E9F7D02E4FF126754A6
:10397E007BFF7A197965900027E0FCA3E0FDA3E0B8
:10398E00FEA3E0F54C8E4B8D4A8C49123E9F7D0274
:10399E007F0A1267547BFF7A19797090002BE0FC36
:1039AE00A3E0FDA3E0FEA3E0F54C8E4B8D4A8C49BF
:1039BE00123E9F7D03E4FF12675490000FE07008E3
:1039CE007BFF7A19797B802190000FE0B401087B90
:1039DE00FF7A197981801290001DE07BFF60067AD4
:1039EE0019798880047A19798E123E9F7D037F069D
:1039FE00126754900010E070087BFF7A197994805A
:103A0E0021900010E0B401087BFF7A19799A801298
:103A1E0090001EE07BFF60067A1979A180047A1966
:103A2E0079A7123E9F7D037F0D12675490000EE022
:103A3E007BFFB401067A1979AD80047A1979B41234
:103A4E003E9F3017332013301267979000001216E6
:103A5E006B90000FE00475F00384AFF0EFF070068A
:103A6E0090001DF0800D90000FE0B4010690001D37
:103A7E007401F07F0A12476C30182A201427900028
:103A8E0010E00475F00384AFF0EFF0700690001EA6
:103A9E00F0800D900010E0B4010690001E7401F04D
:103AAE007F0B12476C201903023BA72015279000AD
:103ABE0027E0FCA3E0FDA3E0FEA3E0FFE4FBFA7920
:103ACE0080783F120D3790002712166B1267979071
:103ADE00000412166B126797C8ECC8C9EDC9CAEE7E
:103AEE00CACBEFCB900004E0FCA3E0FDA3E0FEA365
:103AFE00E02446FFE43EFEE43DFDE43CFCD312151B
:103B0E0075401E900027E0FCA3E0FDA3E0FEA3E0BD
:103B1E00FFE4FBFA7980783F120D379000271216DA
:103B2E006B126797C8ECC8C9EDC9CAEECACBEFCB0A
:103B3E00900004E0FCA3E0FDA3E0FEA3E0242CFF34
:103B4E00EE3401FEE43DFDE43CFCD3121575401E3F
:103B5E00900027E0FCA3E0FDA3E0FEA3E0FFE4FB62
:103B6E00FA79107841120D3790002712166BE4FF88
:103B7E00FE7DC87C42900027E0F8A3E0F9A3E0FAAE
:103B8E00A3E0FB120FCE600C400A900027121677AE
:103B9E0042C800007F0E12476C201A03023C972089
:103BAE001627900027E0FCA3E0FDA3E0FEA3E0FFB4
:103BBE00E4FBFA7980783F120D3390002712166BD2
:103BCE0012679790000412166B126797C8ECC8C95B
:103BDE00EDC9CAEECACBEFCB900004E0FCA3E0FD2A
:103BEE00A3E0FEA3E02446FFE43EFEE43DFDE43CFC
:103BFE00FCD3121575401E900027E0FCA3E0FDA338
:103C0E00E0FEA3E0FFE4FBFA7980783F120D3390DB
:103C1E00002712166B126797C8ECC8C9EDC9CAEE19
:103C2E00CACBEFCB900004E0FCA3E0FDA3E0FEA323
:103C3E00E0242CFFEE3401FEE43DFDE43CFCD31207
:103C4E001575401E900027E0FCA3E0FDA3E0FEA347
:103C5E00E0FFE4FBFA79107841120D339000271241
:103C6E00166BE4FFFEFDFC900027E0F8A3E0F9A33D
:103C7E00E0FAA3E0FB120FCE500A9000271216773F
:103C8E00000000007F0E12476C301911301A0E2002
:103C9E001903301A051255A880F57F012290000FE6
:103CAE00E064026003023D36A3E06402707A900085
:103CBE001DE07074126797900000E0F8A3E0F9A37E
:103CCE00E0FAA3E0FBC3EF9BFFEE9AFEED99FDEC4D
:103CDE0098FCECC0E0EDC0E0EEC0E0EFC0E090007C
:103CEE0015E0FEA3E0FF7C007D64121484CAEECAC8
:103CFE00CBEFCB900013E0FEA3E0FF121484C3EFD2
:103D0E009BFFEE9ACBEFCBFAE4F9F8D0E0FFD0E0D0
:103D1E00FED0E0FDD0E0FCC3121575500B90001ED6
:103D2E007401F07F0B12476C90000FE06402706E0E
:103D3E0090001DE07068126797900000E0F8A3E015
:103D4E00F9A3E0FAA3E0FBC3EF9BFFEE9AFEED9919
:103D5E00FDEC98FCECC0E0EDC0E0EEC0E0EFC0E0A2
:103D6E00900013E0FEA3E0FF7C007D64121484CB70
:103D7E00EFCBCAEECAE4F9F8D0E0FFD0E0FED0E017
:103D8E00FDD0E0FCC3121575501412679790000019
:103D9E0012166B90001D7401F07F0A12476C900092
:103DAE000FE06402707690001DE06401706E126781
:103DBE0097900000E0F8A3E0F9A3E0FAA3E0FBC3BC
:103DCE00EF9BFFEE9AFEED99FDEC98FCECC0E0ED5A
:103DDE00C0E0EEC0E0EFC0E0900011E0FEA3E0FF17
:103DEE007C007D64121484CBEFCBCAEECAE4F9F8E2
:103DFE00D0E0FFD0E0FED0E0FDD0E0FCC3121575A0
:103E0E00501A12679790000012166BE490001DF086
:103E1E00A3F07F0A12476C7F0B12476CA217921306
:0E3E2E00A2189214A2199215A21A92167F00E1
:013E3C002263
:104EC60090000EE064016003025008126797C8EC78
:104ED600C8C9EDC9CAEECACBEFCB900009E0FCA366
:104EE600E0FDA3E0FEA3E02470FFEE3417FEE43DF0
:104EF600FDE43CFCD3121575500302500812679767
:104F060090000912166B900027E0FCA3E0FDA3E0D9
:104F1600FEA3E0FF90031912166B900073E0FCA34A
:104F2600E0FDA3E0FEA3E0FF900033E0F8A3E0F984
:104F3600A3E0FAA3E0FB120FCE60025037E4FFFEB7
:104F46007D5C7C42900019E0F8A3E0F9A3E0FAA3A7
:104F5600E0FB120FCE401D7F337E337DB37C3F9046
:104F66000067E0F8A3E0F9A3E0FAA3E0FB120FCE96
:104F760060194017900319E0FCA3E0FDA3E0FEA32F
:104F8600E0FFE4FBFA798078BF8014900319E0FC17
:104F9600A3E0FDA3E0FEA3E0FFE4FBFAF9783F12ED
:104FA6000D3790031912166BE4FFFE7D887C419045
:104FB6000319E0F8A3E0F9A3E0FAA3E0FB120FCE91
:104FC600600C400A90031912167741880000E4FF2E
:104FD600FEFD7C41900319E0F8A3E0F9A3E0FAA3F3
:104FE600E0FB120FCE500A9003191216774100000B
:104FF600007B017A0079279003191267417F0E1210
:02500600476CF5
:015008002285
:1000A600900008E075F004A42477F9740035F0FA9E
:1000B6007B01E0FF7E00124B72900008E0703D7FEE
:1000C600427E607DD57C3F900077E0F8A3E0F9A3FF
:1000D600E0FAA3E0FB120E287BAE7A47793578C1A9
:1000E600120D378F428E418D408C3F7F007E007D02
:1000F600207C4112526990006312166B900008E052
:10010600640260030201B57B6F7A127983783A90B4
:10011600007FE0FCA3E0FDA3E0FEA3E0FF120F31A9
:1001260090031112166BE4FFFE7D5C7CC3900311F5
:10013600E0F8A3E0F9A3E0FAA3E0FB120D37E4FB35
:10014600FA79937843120E28E4FBFA798C784212F6
:100156000F31E4FBFA798778C3120D379003111239
:10016600166B900311E0FCA3E0FDA3E0FEA3E0FF05
:100176007B007A8079887843120D37900311121626
:100186006BE4FFFEFDFC900311E0F8A3E0F9A3E0A9
:10019600FAA3E0FB120FCE500A9003111216770055
:1001A6000000007B017A00792F90031112674190BD
:1001B6000008E06404705BFFFE7D207C41900087B0
:1001C600E0F8A3E0F9A3E0FAA3E0FB120E289003FF
:1001D6001112166BE4FFFE7D807CC0900311E0F8DF
:1001E600A3E0F9A3E0FAA3E0FB120D37E4FBFA79EA
:1001F600807841120F31E4FBFA79C87842120E2852
:1002060090031112166B7B017A0079199003111273
:100216006741900008E06405705BFFFE7D207C412D
:1002260090008BE0F8A3E0F9A3E0FAA3E0FB120E3E
:100236002890031112166BE4FFFE7D807CC09003AC
:1002460011E0F8A3E0F9A3E0FAA3E0FB120D37E40E
:10025600FBFA79807841120F31E4FBFA7920784075
:10026600120E2890031112166B7B017A00796790A3
:100276000311126741900008E0045407F0E4FFFE02
:100286007D7A7C449000D7E0F8A3E0F9A3E0FAA3D6
:10029600E0FB120E28E4FBFA796078C3120D377B77
:1002A600937A18790478C0120F31E4FBFA798778CB
:1002B60043120D3790031512166BE4FFFEFDFC90FA
:1002C6000315E0F8A3E0F9A3E0FAA3E0FB120FCED2
:1002D600401D7F007EC07D797C44900315E0F8A325
:1002E600E0F9A3E0FAA3E0FB120FCE600C400A90FF
:1002F6000315121677000000007A00791F12673C7A
:10030600E4FFFE7D7A7C449000DBE0F8A3E0F9A3ED
:10031600E0FAA3E0FB120E28E4FBFA796078C31238
:100326000D377B937A18790478C0120F31E4FBFA03
:1003360079877843120D3790031512166BE4FFFE8A
:10034600FDFC900315E0F8A3E0F9A3E0FAA3E0FBB7
:10035600120FCE401D7F007EC07D797C4490031530
:10036600E0F8A3E0F9A3E0FAA3E0FB120FCE600CDD
:10037600400A900315121677000000007A007923D0
:1003860012673CE4FFFE7D7A7C449000DFE0F8A330
:10039600E0F9A3E0FAA3E0FB120E28E4FBFA796089
:1003A60078C3120D377B937A18790478C0120F310F
:1003B600E4FBFA79877843120D3790031512166B12
:1003C600E4FFFEFDFC900315E0F8A3E0F9A3E0FAD4
:1003D600A3E0FB120FCE401D7F007EC07D797C44DA
:1003E600900315E0F8A3E0F9A3E0FAA3E0FB120FEF
:1003F600CE600C400A900315121677000000007BB1
:10040600017A00793B12673EE4FFFE7D7A7C4490D8
:1004160000E3E0F8A3E0F9A3E0FAA3E0FB120E285C
:10042600E4FBFA795578C3120D377B687A91790522
:1004360078C0120F31E4FBFA79877843120D3790B2
:10044600031512166BE4FFFEFDFC900315E0F8A3FE
:10045600E0F9A3E0FAA3E0FB120FCE401D7F007E79
:10046600C07D797C44900315E0F8A3E0F9A3E0FA97
:10047600A3E0FB120FCE600C400A9003151216770C
:10048600000000007B017A00793F12673EE4FFFE20
:100496007D7A7C449000E7E0F8A3E0F9A3E0FAA3B4
:1004A600E0FB120E28E4FBFA796578C3120D377B60
:1004B600B67AF379FD78BF120F31E4FBFA798778C3
:1004C60043120D3790031512166BE4FFFEFDFC90E8
:1004D6000315E0F8A3E0F9A3E0FAA3E0FB120FCEC0
:1004E600401D7F007EC07D797C44900315E0F8A313
:1004F600E0F9A3E0FAA3E0FB120FCE600C400A90ED
:100506000315121677000000007B017A007943126A
:10051600673EE4FFFE7D7A7C449000EBE0F8A3E0C2
:10052600F9A3E0FAA3E0FB120E28E4FBFA7973784C
:10053600C3120D377B877A1679F978BF120F31E42B
:10054600FBFA79877843120D3790031512166BE480
:10055600FFFEFDFC900315E0F8A3E0F9A3E0FAA383
:10056600E0FB120FCE401D7F007EC07D797C44905B
:100576000315E0F8A3E0F9A3E0FAA3E0FB120FCE1F
:10058600600C400A900315121677000000007B01EC
:100596007A00794712673EE4FFFE7D7A7C4490003C
:1005A600EFE0F8A3E0F9A3E0FAA3E0FB120E28E4DB
:1005B600FBFA796478C3120D377BE97A26790178DC
:1005C600C0120F31E4FBFA79877843120D37900396
:1005D6001512166BE4FFFEFDFC900315E0F8A3E090
:1005E600F9A3E0FAA3E0FB120FCE401D7F007EC008
:1005F6007D797C44900315E0F8A3E0F9A3E0FAA323
:10060600E0FB120FCE600C400A900315121677001D
:100616000000007B017A00794B12673EE4FFFE7D05
:100626007A7C449000F3E0F8A3E0F9A3E0FAA3E0B3
:10063600FB120E28E4FBFA796678C3120D377BEEBF
:100646007A7C79FF78BF120F31E4FBFA7987784319
:10065600120D3790031512166BE4FFFEFDFC900396
:1006660015E0F8A3E0F9A3E0FAA3E0FB120FCE40F1
:100676001D7F007EC07D797C44900315E0F8A3E0E1
:10068600F9A3E0FAA3E0FB120FCE600C400A900338
:1006960015121677000000007B017A00794F126769
:1006A6003EE4FFFE7D7A7C449000F7E0F8A3E0F993
:1006B600A3E0FAA3E0FB120E28E4FBFA796678C3FE
:1006C600120D377B687A9179FD78BF120F31E4FB02
:1006D600FA79877843120D3790031512166BE4FFEB
:1006E600FEFDFC900315E0F8A3E0F9A3E0FAA3E011
:1006F600FB120FCE401D7F007EC07D797C449003A7
:1007060015E0F8A3E0F9A3E0FAA3E0FB120FCE6030
:100716000C400A900315121677000000007B017A40
:1007260000795312673EE4FFFEFDFC9000FBE0F803
:10073600A3E0F9A3E0FAA3E0FB120FCE70030208D0
:10074600DF9000FBE0F8A3E0F9A3E0FAA3E0FBE406
:10075600FFFE7D807C3F120F3190031112166B7FD6
:10076600D87E817DF37C3D900311E0F8A3E0F9A3E8
:10077600E0FAA3E0FB120E28900311E0F8A3E0F9DB
:10078600A3E0FAA3E0FB120E28900311E0F8A3E021
:10079600F9A3E0FAA3E0FB120E28900311E0F8A3F8
:1007A600E0F9A3E0FAA3E0FB120E28ECC0E0EDC0EE
:1007B600E0EEC0E0EFC0E07F637EEE7DF27C3F902E
:1007C6000311E0F8A3E0F9A3E0FAA3E0FB120E2878
:1007D600900311E0F8A3E0F9A3E0FAA3E0FB120E00
:1007E60028900311E0F8A3E0F9A3E0FAA3E0FB12D6
:1007F6000E28C8ECC8C9EDC9CAEECACBEFCBD0E00B
:10080600FFD0E0FED0E0FDD0E0FC120D33ECC0E0FE
:10081600EDC0E0EEC0E0EFC0E07F7F7E6A7D467C03
:1008260041900311E0F8A3E0F9A3E0FAA3E0FB127C
:100836000E28900311E0F8A3E0F9A3E0FAA3E0FB89
:10084600120E28D0E0FBD0E0FAD0E0F9D0E0F812A2
:100856000D37ECC0E0EDC0E0EEC0E0EFC0E07F3F5A
:100866007EB57D0D7C42900311E0F8A3E0F9A3E08C
:10087600FAA3E0FB120E28C8ECC8C9EDC9CAEECA35
:10088600CBEFCBD0E0FFD0E0FED0E0FDD0E0FC1215
:100896000D33E4FBFA79227842120D3790031512D4
:1008A600166BE4FFFEFDFC900315E0F8A3E0F9A348
:1008B600E0FAA3E0FB120FCE401F7F007EC07D79D9
:1008C6007C44900315E0F8A3E0F9A3E0FAA3E0FB6B
:1008D600120FCE600E400C800090031512167700A2
:1008E6000000007B017A00795712673EE4FFFEFDA7
:1008F600FC9000FFE0F8A3E0F9A3E0FAA3E0FB1206
:100906000FCE7003020AA59000FFE0F8A3E0F9A35A
:10091600E0FAA3E0FBE4FFFE7D807C3F120F3190FE
:10092600031112166B7FCE7EAA7D0F7C3E900311BB
:10093600E0F8A3E0F9A3E0FAA3E0FB120E28900387
:1009460011E0F8A3E0F9A3E0FAA3E0FB120E289069
:100956000311E0F8A3E0F9A3E0FAA3E0FB120E28E6
:10096600900311E0F8A3E0F9A3E0FAA3E0FB120E6E
:1009760028ECC0E0EDC0E0EEC0E0EFC0E07F7C7E9A
:10098600F27D147C40900311E0F8A3E0F9A3E0FAAD
:10099600A3E0FB120E28900311E0F8A3E0F9A3E010
:1009A600FAA3E0FB120E28900311E0F8A3E0F9A3E6
:1009B600E0FAA3E0FB120E28C8ECC8C9EDC9CAEEDE
:1009C600CACBEFCBD0E0FFD0E0FED0E0FDD0E0FC1C
:1009D600120D33ECC0E0EDC0E0EEC0E0EFC0E07F0A
:1009E6005E7EBA7D7B7C41900311E0F8A3E0F9A31B
:1009F600E0FAA3E0FB120E28900311E0F8A3E0F959
:100A0600A3E0FAA3E0FB120E28D0E0FBD0E0FAD078
:100A1600E0F9D0E0F8120D37ECC0E0EDC0E0EEC032
:100A2600E0EFC0E07F547EE37D3A7C42900311E024
:100A3600F8A3E0F9A3E0FAA3E0FB120E28C8ECC87D
:100A4600C9EDC9CAEECACBEFCBD0E0FFD0E0FED0ED
:100A5600E0FDD0E0FC120D33E4FBFA795A7842123D
:100A66000D3790031512166BE4FFFEFDFC9003157F
:100A7600E0F8A3E0F9A3E0FAA3E0FB120FCE401FD3
:100A86007F007EC07D797C44900315E0F8A3E0F9F1
:100A9600A3E0FAA3E0FB120FCE600E400C8000909C
:100AA6000315121677000000007B017A00795B12AD
:100AB600673EE4FFFEFDFC900103E0F8A3E0F9A326
:100AC600E0FAA3E0FB120FCE7003020C6C90010358
:100AD600E0F8A3E0F9A3E0FAA3E0FBE4FFFE7D80E3
:100AE6007C3F120F3190031112166B7F127E147D1C
:100AF6007F7C3E900311E0F8A3E0F9A3E0FAA3E0BF
:100B0600FB120E28900311E0F8A3E0F9A3E0FAA384
:100B1600E0FB120E28900311E0F8A3E0F9A3E0FA37
:100B2600A3E0FB120E28900311E0F8A3E0F9A3E07E
:100B3600FAA3E0FB120E28ECC0E0EDC0E0EEC0E048
:100B4600EFC0E07F017EDE7D8A7C40900311E0F8F5
:100B5600A3E0F9A3E0FAA3E0FB120E28900311E04C
:100B6600F8A3E0F9A3E0FAA3E0FB120E2890031124
:100B7600E0F8A3E0F9A3E0FAA3E0FB120E28C8EC24
:100B8600C8C9EDC9CAEECACBEFCBD0E0FFD0E0FEB4
:100B9600D0E0FDD0E0FC120D33ECC0E0EDC0E0EE9D
:100BA600C0E0EFC0E07F087EAC7DE97C4190031198
:100BB600E0F8A3E0F9A3E0FAA3E0FB120E28900305
:100BC60011E0F8A3E0F9A3E0FAA3E0FB120E28D0A7
:100BD600E0FBD0E0FAD0E0F9D0E0F8120D37ECC037
:100BE600E0EDC0E0EEC0E0EFC0E07F377E097DAA11
:100BF6007C42900311E0F8A3E0F9A3E0FAA3E0FB3E
:100C0600120E28C8ECC8C9EDC9CAEECACBEFCBD0C4
:100C1600E0FFD0E0FED0E0FDD0E0FC120D337BCD4E
:100C26007ACC79BA7842120D3790031512166BE416
:100C3600FFFEFDFC900315E0F8A3E0F9A3E0FAA39C
:100C4600E0FB120FCE401F7F007EC07D797C449072
:100C56000315E0F8A3E0F9A3E0FAA3E0FB120FCE38
:100C6600600E400C800090031512167700000000FD
:100C76007B017A00795F12673EE4FFFE7DC07C400F
:100C8600900107E0F8A3E0F9A3E0FAA3E0FB120E57
:100C96002890031112166B7B717A3D79EA784090A1
:100CA6000311E0FCA3E0FDA3E0FEA3E0FF120F3179
:100CB600C8ECC8C9EDC9CAEECACBEFCBE4FFFE7DCE
:100CC600807C3F120D33E4FBFA79C87842120E2875
:100CD60090031112166BE4FFFEFDFC900311E0F881
:100CE600A3E0F9A3E0FAA3E0FB120FCE500A9003AB
:100CF60011121677000000007B017A007933900309
:100D0600111267411255A812332D124EC678277C50
:100D1600017D017B017A00790D7E017F1A1213E4B1
:090D260090000DE0B47B0280FE98
:010D2F0022A1
:1066E40020202020557067726164696E6700202045
:0E66F40020204669726D776172652E2E2E0091
:10608D000189000108FF42024BFFFF44024D000051
:02609D00000001
:1042AC00E47889F612678975840F75E104E4F5E208
:1042BC0075E344F58475B7B075840F438901758D2A
:1042CC0001758F01758E04F53DF53E053EE53E709A
:1042DC0002053D640F453D70F2438902E58930E4E7
:1042EC00FB758A83759702126132E4FF126702E450
:1042FC00F53DF53E7D01AF3E126657053EE53E703D
:10430C0002053DC39403E53D940040E8E4F520C26A
:10431C001EC21BC222C221C2207889F6C2857882B5
:10432C00F67880F618F67887F6F53DF53E7451254B
:10433C003EF582E43402F583E4F0053EE53E70027E
:10434C00053D6440453D70E5E4F53DF53E74912531
:10435C003EF582E43402F583E4F0053EE53E70025E
:10436C00053D6440453D70E5E4F584E5EF20E10C46
:10437C00E5EF5408D394004003D38001C392037D2E
:10438C0008E4FF1263977D087F01126397125F2286
:10439C00E47885F6787DF6AB76AA77A978787DE611
:1043AC00FF75F01FA4F58285F083121423FE788527
:1043BC0026F6EE6005787D0680DDEFD3940040286C
:1043CC00AB76AA77A97890000D1216C97455121401
:1043DC005012140A64556002D22074AA121450129E
:1043EC00140A64AA6002D22012566A8F3CE53C2063
:1043FC00E037C21D74FFF509F50AF50BF50CE4F571
:10440C000DF50EFE7F10FDFB7A00790F1218087562
:10441C0049FF754A19754BBB754C00754D107B00E7
:10442C007A00790F1262F48002D21DE53C30E10370
:10443C000244E3C21FE4F53DF53EAB76AA77A978BA
:10444C00853E82853D83741F1216A81214237003B7
:10445C000244DFAE3DAF3E7C007D1F121484E92F79
:10446C00F9EA3EFA90000412142320E25BE4F53BD7
:10447C00E53BC378A1965050AB76AA77A978853ED8
:10448C0082853D83741F1216A8121423FF7E00C070
:10449C0006C0077F00C007AE3DAF3E7C007D1F12FB
:1044AC001484E92FF9EA3EFA90000D1216C97885AA
:1044BC00E6853BF0A429F9EA35F0FAD005D007D00F
:1044CC0006121808053B80A8053EE53E7002053D26
:1044DC000244467F018004D21FE4FF124D3F30039B
:1044EC00057886068004E47886F67886E6750D00F5
:1044FC00F50EE4F53DF53E7A007B967D03AF3E125A
:10450C005EA9053EE53E7002053DC39403E53D946E
:03451C000040E478
:01451F002279
:0567C9007887E6FF22C5
:0300230002538005
:10538000C0E0C0F0C083C082C0D075D000C000C0F3
:1053900001C002C003C004C005C006C00730993F69
:1053A000C2997880067980E778826670167880F6F0
:0253B000D21C0D
:0D53B20075260A75271300D527FCD526F6B1
:0453BF00C285801C07
:0D53C30075261475271300D527FCD526F696
:1053D0007880E62491F582E43402F583E0F59920A3
:1053E0009803025479209A08201E05C29802547529
:1053F000C29A787FE6062451F582E43402F583E50B
:1054000099F0C298E6FFB40112900251E0FE7003D9
:10541000F68066EE540724027888F6EFB4020D7821
:1054200088E6B40907900252E02403F6787FE6FF8D
:10543000B4400476008042EFC3788896403B787F82
:10544000E624FFFDE434FFFC7B017A027951125B14
:105450008A787FE62450F582E43402F583E06F60B9
:05546000047600801439
:0D54650075261475271300D527FCD526F6F3
:10547200122B92787F7600D007D006D005D004D0C8
:1054820003D002D001D000D0D0D082D083D0F0D0CF
:02549200E03206
:105E2D00900252E075F01FA4AB762578F9E5773531
:105E3D00F0FA90000D1216C97887E6FF7885E68F87
:105E4D00F0A4252AF582E435F0F583121423FF7BA7
:055E5D00007A00792825
:105E62008F358B368A378938E4F584EA494B601CD2
:105E7200AB36AA37A93812140AFFE535FD7C0012A9
:0C5E82000003AB36AA37A938EF12145009
:0D5E8E00753914753A1300D53AFCD539F674
:0E5E9B008535997F0112662E3099FDC299223D
:0B66C500E4F5847882EFF6C21CD28559
:0D66D00075351475361300D536FCD535F63A
:0766DD00900291E0F5992203
:10648600C9EFC9E964017028EDC39B403478A1E6E1
:10649600FFEB2FFFE433FEEDC39FEE6480F87480BC
:1064A60098501ED21EC3ED9B7887F678817601221E
:1064B600B90214ED6B700AD21E7887F678817602DF
:0864C60022C21EE47881F622D7
:1060D100C9EFC9BAFF15BBFF12ED6B7002EC6A7014
:1060E10049D21E7887F67881E9F622E964017025A4
:1060F100C3ED9BEC9A401C78A1E62BFFE43AFEC36A
:10610100ED9FEC9E500DD21EC3ED9B7887F67881F2
:106111007601228015B90218ED6B7002EC6A700AE3
:10612100D21E7887F67881760222C21EE47881F643
:01613100224B
:102B9200900251E0FF54F8F529E4F584EF1216F99A
:102BA2002BDF092BEB0A2BFB102C04112C14122CFB
:102BB20028192C3D1A2C5F202C68282D07292E0954
:102BC200332E3B372E67392E77412E82492E8C5079
:102BD2002ED4612DD3702ECC9800002F0490025277
:102BE200E0FDE50AFB7F018023900252E0FCA3E0B6
:102BF200FDAB0AAA097F018027D21E7881760302E3
:102C02002F04900252E0FDE50CFB7F021264860263
:102C12002F04900252E0FCA3E0FDAB0CAA0B7F0252
:102C22001260D1022F04900252E0FDE50AFB7F01FF
:102C3200126486201E03022F048017900252E0FCC9
:102C4200A3E0FDAB0AAA097F011260D1201E030294
:102C52002F049002917478F07F01022F01E4F58431
:102C620075EF10022F04C2ACE4F528D285FB7A007E
:102C720079287F7F125E627B007A0079287F1812A2
:102C82005E627B007A0079287F04125E62787DE6BC
:102C9200125E5B7B007A007928AF09125E627B00CC
:102CA2007A007928AF0A125E627B007A007928AF37
:102CB2000B125E627B007A007928AF0C125E627B97
:102CC200007A007928AF0D125E627B007A007928C3
:102CD200AF0E125E62E4F52A740F252AF8E6125E40
:102CE2005B052AE52AC3941040EE7B007A00790046
:052CF200AF28125E6234
:0D2CF70075330A75341300D534FCD533F65F
:102D0400022DBE900252E0FFC3787D964003022D4F
:102D1400C5EF75F01FA42578F9E57735F085763091
:102D2400F5318932C2ACE4F528D285FB7A007928E2
:102D34007F7F125E627B007A0079287F0D125E62CB
:102D4400AB30AA31A93212140A125E5BAB30AA313D
:102D5400A932900001125E58AB30AA31A93290001A
:102D640002125E58AB30AA31A932900003125E58A9
:102D7400AB30AA31A932900004125E58E4F52AABB4
:102D840030E5322405F9E43531FA7E00E9252AF9E3
:102D9400EE3AFA12140A125E5B052AE52AC3940875
:0D2DA40040DD7B007A007900AF28125E62EE
:0D2DB10075330A75341300D534FCD533F6A4
:102DBE00C285D2AC022F049002917478F0E4A3F095
:102DCE007F02022F011267A4789612165F9002916D
:102DDE00747CF07896E6A3F008E6A3F008E6A3F07C
:102DEE0008E6A3F07C007D057B017A027991125BE7
:102DFE008A900296EFF07F06022F01900252E0FFBA
:102E0E00B4010BA3E0F509A3E0F50A022ECCEFB452
:102E1E000209900253E0F509022ECC900252E0B462
:102E2E000308A3E0F50BA3E0F50C022ECCE4F52A83
:102E3E00900252E0FFE52AC39F501C7453252AF5D9
:102E4E0082E43402F583E0FF740F252AF8C6EFC63C
:102E5E00052AE52AB410D980657A007B327D017887
:102E6E0087E6FF125EA9022F04900252E024FF9221
:102E7E0002022F04900252E024FF9201807878879C
:102E8E00E66005752C02800B202105752C0380034E
:102E9E00752C019002917479F0A3E52CF07C007DE5
:102EAE00027B017A027991125B8A900293EFF07F96
:102EBE00031266C5E52C6401703CD2228002D21B3F
:102ECE00788976F180307A007B327D017F00125E48
:102EDE00A99002917479F0900252E0900292F07CE7
:102EEE00007D027B017A027991125B8A900293EF48
:102EFE00F07F031266C5E52964A0600302310090DD
:102F0E000251E064A16003023003A3E0C3787D9612
:102F1E004003022FF8AB76AA77A978E0FF75F01F71
:102F2E00A4F58285F083121423F52CEF75F01FA4FF
:102F3E0029F9EA35F0FA90000412142330E23790A2
:102F4E000252E01267C48F2C900291747FF0A3E5B9
:102F5E002CF02402FDE433FC7B017A027991125BA2
:102F6E008A7493252CF582E43402F583EFF0E52C78
:102F7E002403FF0230FD900252E0FF1267C4C2AC80
:102F8E00E4F528D285E52CD39406402B7B007A00FD
:102F9E0079287F7F125E627B007A007928AF2C122F
:102FAE005E62E4F52AE52AC3952C5007125E2D05C4
:102FBE002A80F2052C8018E52C2478125E5BE4F54D
:102FCE002AE52AC3952C5007125E2D052A80F27B26
:0A2FDE00007A007900AF28125E624D
:0D2FE80075330A75341300D534FCD533F66B
:102FF5000230EF9002917478F07F010230FD90026B
:1030050051E064A26003023100787DE6FFA3E0FE93
:10301500C39F40030230F5A3E0FDC39F4003023088
:10302500F5EEC39D40030230F5900252E0F52AE427
:10303500F52C900253E0FFE52AD39F5021AF2A12C9
:1030450067C4AB76AA77A97875F01FE52AA4F5823F
:1030550085F083121423252CF52C052A80D4C2ACC7
:10306500E4F528D285FB7A0079287F7F125E627BA2
:10307500007A007928AF2C125E62900252E0F52AA0
:10308500900253E0FFE52AD39F5047E4F52BAB763A
:10309500AA77A97875F01FE52AA4F58285F0831231
:1030A5001423FFE52BC39F5025E52A75F01FA4299E
:1030B500F9EA35F0FA90000D1216C97887E6FF781F
:1030C50085E68FF0A4252B125E51052B80C0052ABD
:0D30D50080AE7B007A007900AF28125E62A9
:0D30E20075330A75341300D534FCD533F670
:1030EF00C285D2AC800B9002917478F07F0112668A
:1030FF00C5E5296458704DFA7B327D017887E6FF6C
:10310F00125EA9753801753902753A927B017A0200
:10311F00795212657F8F2CE52C2478900291F0EF75
:10312F002401FDE433FC7B017A027991125B8A74EE
:10313F0092252CF582E43402F583EFF0E52C24027E
:10314F00FF1266C5E52964806009E529648860037C
:10315F0002332C7881E6B4010F7A007B327D01783F
:10316F0087E6FF125EA9801AE4F52AE52AC378A143
:10317F0096500F7A007B327D01AF2A125EA9052A85
:10318F0080E9900251E05407F52CB4070A752B0122
:10319F00A3E0F52CA38006E4F52B900252E0F52D69
:1031AF00152CE52DC3787D964003023300AB76AA2C
:1031BF0077A97875F01FE52DA4F58285F083121499
:1031CF0023FFE52CD39F40028F2C7881E6B40109B1
:1031DF007887E6F52FF52E8009E4F52E78A1E61411
:1031EF00F52F7887A62E7887E6D3952F40030232E6
:1031FF00D8E4F52AE52AC3952C40030232CDE52DFC
:10320F0075F01FA4AB762578F9E57735F0FA9000C5
:10321F000412142330E2030232C890000112142367
:10322F0064387041E52CD394044011E52B252A24F2
:10323F0053F582E43402F583E0FD805E787FE6C3C8
:10324F00952AFFE49400FE744F2FF58274023EF529
:10325F0083E0FDE52D75F01FA4AB762578F9E577B2
:10326F0035F0FA8035AB76AA77A97875F01FE52D82
:10327F00A4F58285F083121423FFC3787FE69F2580
:10328F002A252B2450F582E43402F583E0FDE52D49
:10329F0075F01FA429F9EA35F0FA90000D1216C93E
:1032AF007887E6FF7885E68FF0A4FFE52A2FF58271
:1032BF00E435F0F583ED121462052A023203AF2DC7
:1032CF0012476C7887060231F57887A62EE52D75A3
:1032DF00F01FA4AB762578F9E57735F0FA90000466
:1032EF0012142330E503852D08E5296488702E809C
:1032FF0010E52DB4FF27900253E0F520E529B4889F
:10330F001C9002917478F0787FE62450F582E434B3
:0D331F0002F583E0900292F07F021266C575
:01332C00227E
:09629E0090001C1214F7FFAEF091
:1062A7008E408F4190024BE065407004A3E065414A
:1062B700603A900241740AF0E540A3F0E541A3F08B
:1062C7007C007D037B017A027941125B8A9002444C
:1062D700EFF07B017A0279417547017D047C00125A
:0D62E7005AFD90024BE540F0A3E541F02286
:03634600CCEECCCE
:10634900900241741AF0A3ECF0EFA3F07C007D03F6
:106359007B017A027941125B8A900244EFF07B015A
:106369007A0279417547017D047C00125AFD7B014F
:106379007A0279417D0A7C00125A66EF7002FF2287
:0D638900900241E0647860037F00227F01F4
:0163960022E4
:1065AC007A007B327D017F01125EA974FF90024B51
:1065BC00F0A3F07F0A900241E4F0A3DFFC7B017AA8
:0D65CC000279417547017D0A7C00025AFDED
:10513E00E4F53BE53BC3787D964003025268E53BC0
:10514E0075F01FA4AB762578F9E57735F0FA900067
:10515E000412142320E40302526312629E90024151
:10516E0074A1F0E53B75F01FA4AB762578F9E577D1
:10517E0035F0FA90001E121423900242F07C007D4E
:10518E00027B017A027941125B8A900243EFF07B37
:10519E00017A027941E4F5477D03FC125AFD7B0149
:1051AE007A0279417D647C00125A668F3CE53CC3DD
:1051BE0094025002804DE53C2476FF900241E06F50
:1051CE006002803FAB76AA77A97875F01FE53BA405
:1051DE00F58285F083121423FFE53C24FE6F6002F6
:1051EE008021E53C24FFFDE434FFFC7B017A02794B
:1051FE0041125B8A7440253CF582E43402F583E06B
:10520E006F6007AF3B1265AC804BC2AFAB76AA772F
:10521E00A97875F01FE53BA4F58285F0831214235F
:10522E00FF7E00EEC0E0EFC0E0E53B75F01FA42965
:10523E00F9EA35F0FA90000D1216C9C8E9C8CCEAA1
:10524E00CCCDEBCD7B017A027942D0E0FFD0E0FEEF
:0A525E001213E4D2AF053B025141E8
:015268002223
:025CA2008F3E33
:105CA400EF75F01FA4AB762578F9E57735F0FA1295
:105CB400629EAB76AA77A97875F01FE53EA4F582BB
:105CC40085F083121423F53F2481900241F0E53ED0
:105CD40075F01FA429F9EA35F0FA90001E12142376
:105CE400900242F0AF3F7E0090000D1216C9784337
:105CF4007C027D011213E4E53F2402FDE433FC7BC6
:105D0400017A027941125B8A7443253FF582E434B7
:105D140002F583EFF07B017A027941E53F2403FD2C
:095D2400E433FCE4F547025AFDEA
:1064CE00126797C8ECC8C9EDC9CAEECACBEFCB901C
:1064DE00024DE0FCA3E0FDA3E0FEA3E0240AFFE4EE
:1064EE003EFEE43DFDE43CFCD3121575400C12510A
:1064FE003E12679790024D12166BE508F46008AFD6
:08650E0008125CA27508FF22CF
:10F000007889E664F1600302F5E6301CFDC2AF7555
:10F0100084015398FC75FFDE75FFADE4F541F540C2
:10F02000E4F58420982EE4F545F546209822C3E5C2
:09F03000469488E545941350173D
:0DF03900754B0A754C1300D54CFCD54BF6F9
:10F046000546E54670DF054580DBB2A080CF859991
:10F0560040C298E540641A600302F126F545F5467C
:0EF06600209822C3E5469488E5459413501780
:0DF07400754B0A754C1300D54CFCD54BF6BE
:10F081000546E54670DF054580DB3098928599415C
:10F09100C298E4F545F546209822C3E5469488E5F3
:05F0A100459413501717
:0DF0A600754B0A754C1300D54CFCD54BF68C
:10F0B3000546E54670DF054580DB20980302F02016
:10F0C300859941C298E4F545F546209822C3E54663
:08F0D3009488E54594135017E1
:0DF0DB00754B0A754C1300D54CFCD54BF657
:10F0E8000546E54670DF054580DB20980302F020E1
:09F0F800859941C298D285C299A4
:0DF10100754B14754C1300D54CFCD54BF626
:06F10E007599783099FDAF
:0DF11400754B0A754C1300D54CFCD54BF61D
:10F12100C28502F5D8E5406450600302F1B6F545A9
:10F13100F546209822C3E5469488E5459413501777
:0DF14100754B0A754C1300D54CFCD54BF6F0
:10F14E000546E54670DF054580DB20980302F0207A
:09F15E00859941C298D285C2993D
:0DF16700754B14754C1300D54CFCD54BF6C0
:08F174007599793099FDC299EB
:0DF17C00754B14754C1300D54CFCD54BF6AB
:08F189007599013099FDC2994E
:0DF19100754B14754C1300D54CFCD54BF696
:06F19E00E4F5993099FD33
:0DF1A400754B0A754C1300D54CFCD54BF68D
:0FF1B100C28502F5D8E5406401703ED285C2994F
:0DF1C000754B14754C1300D54CFCD54BF667
:08F1CD007599783099FDC29993
:0DF1D500754B14754C1300D54CFCD54BF652
:06F1E200E4F5993099FDEF
:0DF1E800754B0A754C1300D54CFCD54BF649
:10F1F500C28502F5D8E5406402600302F2BCF5451C
:10F20500F546209822C3E5469488E54594135017A2
:0DF21500754B0A754C1300D54CFCD54BF61B
:10F222000546E54670DF054580DB20980302F020A5
:10F23200859941C298E4F542E54113B392A0E541B4
:10F2420025E0FEC3E49400EE94F0502AE5417F00ED
:10F2520025E0FEC394E0501EE54120E01FE4F58462
:10F2620043B701758F038E478F488F828E83F05389
:10F27200B7F0F58F80037542FFE4F584D285C29919
:0DF28200754B14754C1300D54CFCD54BF6A4
:08F28F007599783099FDC299D0
:0DF29700754B14754C1300D54CFCD54BF68F
:06F2A4008542993099FD3E
:0DF2AA00754B0A754C1300D54CFCD54BF686
:10F2B700C28502F5D8E5406403600302F407F5450B
:10F2C700F546209822C3E5469488E54594135017E0
:0DF2D700754B0A754C1300D54CFCD54BF659
:10F2E4000546E54670DF054580DB20980302F020E3
:10F2F400859941C298E4F545F546209822C3E54630
:08F304009488E54594135017AD
:0DF30C00754B0A754C1300D54CFCD54BF623
:10F319000546E54670DF054580DB20980302F020AD
:10F32900859943C298E5411392A0E54125E0FEC3C2
:10F33900E49400EE94F0400302F020E5417D0025BD
:10F34900E0FCC394E0400302F020E4F58443B701F4
:10F35900758F01E54375F020A42DFFE5F03CF547D5
:10F369008F48E4F584F544E544C394205048E4F516
:10F3790045F546209822C3E5469488E545941350FF
:01F38900176C
:0DF38A00754B0A754C1300D54CFCD54BF6A5
:10F397000546E54670DF054580DB20980302F0202F
:10F3A7000548E548AE477002054714F5828E83E5A8
:10F3B70099F0C298054480B1E4F58453B7F0F58F0E
:06F3C700F584D285C29915
:0DF3CD00754B14754C1300D54CFCD54BF658
:08F3DA007599783099FDC29984
:0DF3E200754B14754C1300D54CFCD54BF643
:06F3EF00E4F5993099FDE0
:0DF3F500754B0A754C1300D54CFCD54BF63A
:10F40200C28502F5D8E5406404600302F4B7F5450D
:10F41200F546209822C3E5469488E5459413501793
:0DF42200754B0A754C1300D54CFCD54BF60C
:10F42F000546E54670DF054580DB20980302F02096
:10F43F00859941C298E54125E0F549754A00E4F503
:10F44F0042F545F546054AE54AAE497002054914AD
:10F45F00F5828E83E4932542F5420546E546700218
:0EF46F0005457004E545640270DBD285C29944
:0DF47D00754B14754C1300D54CFCD54BF6A7
:08F48A007599783099FDC299D3
:0DF49200754B14754C1300D54CFCD54BF692
:06F49F008542993099FD41
:0DF4A500754B0A754C1300D54CFCD54BF689
:10F4B200C28502F5D8E5406405600302F5CDF54545
:10F4C200F546209822C3E5469488E54594135017E3
:0DF4D200754B0A754C1300D54CFCD54BF65C
:10F4DF000546E54670DF054580DB20980302F020E6
:10F4EF00859941C298E4F545F546209822C3E54633
:08F4FF009488E54594135017B1
:0DF50700754B0A754C1300D54CFCD54BF626
:10F514000546E54670DF054580DB20980302F020B0
:09F52400859943C298D285C29971
:0DF52D00754B14754C1300D54CFCD54BF6F6
:08F53A0075997F3099FDC2991B
:0DF54200754B14754C1300D54CFCD54BF6E1
:10F54F007599203099FDE54125E0FCE54375F020E4
:10F55F00A42400FFE5F03CF5498F4AE4F542F54459
:02F56F00C2993F
:0DF57100754B14754C1300D54CFCD54BF6B2
:10F57E00854A82854983E493F5993099FD054AE5DC
:10F58E004AAE497002054914F5828E83E4932542F2
:0BF59E00F5420544E544B420C8C299C2
:0DF5A900754B14754C1300D54CFCD54BF67A
:06F5B6008542993099FD29
:0DF5BC00754B0A754C1300D54CFCD54BF671
:10F5C900C285800BE540B40606E4F58475EF10E5C5
:0DF5D900406407600302F0207889F6D2AF8D
:01F5E6002202
:100026007F0012662E201D0B7A007B327D017F0039
:10003600125EA930200B7A007B1E7D017F00125EC6
:10004600A9301B193021167A007B327D017887E6AC
:10005600FF125EA9C21B12588DD21DD21F30222A52
:10006600302127C2221267B1E4FDFF1267547BFFDD
:100076007A6679E41266047D01E4FF1267547BFF19
:100086007A6679F212660412F000126797E47B2C06
:0D0096007A01F9F8C31215755002D221222B
:0E677B001242AC1200261264CE1200A680F567
:10549400005EBCE2613FDD83C29C7E20A3FD1F4110
:1054A4009DC3217FFCA2401E5F01E3BD3E6082DC00
:1054B400237D9FC1421CFEA0E1BF5D0380DE3C62F0
:1054C400BEE0025CDF81633D7C22C09E1D43A1FFE0
:1054D4004618FAA427799BC584DA3866E5BB5907D0
:1054E400DB856739BAE406581947A5FB7826C49AC0
:1054F400653BD987045AB8E6A7F91B45C6987A24B0
:10550400F8A6441A99C7257B3A6486D85B05E7B99F
:105514008CD2306EEDB3510F4E10F2AC2F7193CD8F
:10552400114FADF3702ECC92D38D6F31B2EC0E507F
:10553400AFF1134DCE90722C6D33D18F0C52B0EE6F
:10554400326C8ED0530DEFB1F0AE4C1291CF2D735F
:10555400CA947628ABF517490856B4EA6937D58B4F
:105564005709EBB536688AD495CB2977F4AA48163F
:10557400E9B7550B88D6346A2B7597C94A14F6A82F
:10558400742AC896154BA9F7B6E80A54D7896B351F
:10559400000000002B6096CBDDEE002C96CBDDE501
:0455A400EEF7FAFD27
:05609F00C1AD016B0A18
:105B8A00157C157CA87CECF608EDF6157C157C15C1
:105B9A007CA87CC6EBC608C6EAC608C6E9C6E57C88
:045BAA0024FCF57C66
:105BAE00F80808E4F6A87CF608F6E57C2407F9A8C0
:105BBE007CE6FE08E6FFC3099719E76480F8EE64F9
:105BCE0080985037E57C2404F8CBE6CB08E6FA083B
:105BDE00E6F98F828E83121423A87C080866FFE5EF
:105BEE007C2403F8EFF6E690549493A87C0808F60C
:105BFE00A87C0806E61870B20680AFA87C0808E6F6
:015C0E00FF96
:075C0F00E57C2409F57C226D
:07000300ED6F90549493FF90
:01000A0022D3
:0300A3000263E80D
:1063E800C0E0C083C082C0D0EEC0E0EFC0E0E59856
:1063F80030E1055398FDD22DE59830E024E5692475
:1064080001FFE433FEEF64404E70028011AF69056E
:106418006974D12FF582E43402F583E599F0539835
:10642800FED0E0FFD0E0FED0D0D082D083D0E032E2
:0A5AFD008B428A4389448C458D4694
:105B0700E4F569758401D284E54724FF929BE4F5A7
:105B170048C3E5489546E5456480F8748098505E2B
:025B2700C22D8D
:0D5B2900754914754A1300D54AFCD549F69C
:105B3600E54624FFFFE54534FFFEEF65487001EEBC
:105B4600701EC2ACAB420544E544AA43700205434D
:105B560014F912140AF599302DFDC284D2AC8016C0
:105B6600AB420544E544AA437002054314F91214F6
:105B76000AF599302DFD7F0112662E05488093C2E5
:035B860084AF46A3
:015B890022F9
:0A5A66008B3D8A3E893F8C408D4144
:105A70001267978F468E458D448C43E4F54212673A
:105A800097C3EF9546FFEE9545FEED9544FDEC95E9
:105A900043FCE47B01FAF9F8C312157550037F004B
:105AA00022E569D39400404E9002D1E0FEB4780321
:105AB0007F0122EE54F8647860037F00229002D1C7
:105AC000E054072402F5426569702BD3E5699541DE
:105AD000E5406480F87480984006AE40AF41800491
:105AE000AF697E00A83FAC3EAD3D7B017A0279D123
:0D5AF0001213E4AF42227F0112662E808166
:0667BE00E4F569D22D2272
:10639700EF7025F5847598D0F584759115F584759A
:1063A700C90875CBFFED90559393F5CA75C804E4FA
:1063B700F584D2ACC2BC80267584017598D0E4F50B
:1063C70084E589540F4420F589758E02ED90559D1B
:1063D70093F58DD28E43E74043F7401267BED2AFA5
:0163E7002293
:10613200D2AFD2A9D2BBE4F584E589540F4401F56C
:1061420089758E02758CAFE4F58AD28CF571F57083
:10615200F56FF56EF575F574F573F572756A64FF92
:10616200EF25E025E0248AF8E4F6EF25E025E02497
:106172008BF8E4F6EF25E025E0248CF8E4F6EF2531
:0C618200E025E0248DF8E4F60FBF03D404
:01618E0022EE
:02593000157CE4
:10593200A87CE4F6A87CE6FFC3940340030259C99D
:10594200EF25E025E0248DF8E6FFD394004052A82D
:105952007CE625E025E0248BF8E67045EF30E01583
:10596200A87CE6FF25E025E0248DF8E6D3940140EB
:10597200047D0180067D00A87CE6FF1261ECA87C14
:10598200E6FF25E025E0248DF816E66014EF25E019
:1059920025E0248CF8E6FEEF25E025E0248BF8EEE6
:1059A200F6A87CE625E025E0248BF8E6600116A83F
:1059B2007CE6FF25E025E0248DF8E67004FD126107
:0759C200ECA87C0602593637
:0359C900057C2238
:03000B00025DAFE4
:105DAF00C0E0C0F0C083C082C0D0E8C0E0E9C0E06E
:105DBF00EAC0E0EBC0E0ECC0E0EDC0E0EEC0E0EF29
:105DCF00C0E0758CAFE5712401F571E43570F570A5
:105DDF00E4356FF56FE4356EF56ED56A18E5752409
:105DEF0001F575E43574F574E43573F573E43572C4
:105DFF00F572756A641259301266A5D0E0FFD0E0D3
:105E0F00FED0E0FDD0E0FCD0E0FBD0E0FAD0E0F92E
:0E5E1F00D0E0F8D0D0D082D083D0F0D0E032E6
:10665700157CA87CEDF6157CA87CEFF6A87CE6FFF8
:10666700C39403500D08E6FEEF25E025E0248AF8E1
:07667700EEF6057C057C2214
:105EA900157C157CA87CEAF608EBF6157CA87CED38
:105EB900F6157CA87CEFF6A87CE6FFC39403505244
:105EC900EF25E025E0248DF8E67047A87CE6FB2560
:105ED900E025E0248BF8E67039A87C08E625E00483
:105EE900FFA87CE6FA25E025E0248DF8EFF6A87CEA
:105EF9000808E6FE08E6FF7C007D0A121496EA25EA
:105F0900E025E0248CF8EFF6EB25E025E0248BF87A
:095F1900E4F6E57C2404F57C2289
:1061EC00157CA87CEDF6157CA87CEFF6A87CE6FF68
:1061FC00C39403501CEF25E025E0248AF8E66011D7
:10620C00A87C08E670047F0180027F00A87C08EF60
:10621C00F6A87CE6700608E624FF92A0A87CE6FFB0
:10622C00B4010608E624FF9286EFB40208A87C08A5
:0A623C00E624FF9287057C057C2212
:0C679700C2AFAF71AE70AD6FAC6ED2AF90
:0167A30022D3
:0C67A400C2AFAF75AE74AD73AC72D2AF73
:0167B00022C6
:10662E00157CA87CEFF6A87CE67004F56CF56D3051
:10663E002B14E56B75F064A4FFC3E56D9FE56C95B7
:09664E00F0500375FFA5057C2244
:10670200D22BE4F56CF56DEF6004F56B8003756BCD
:0E6712000A75FF0775FFA5E4F58475EF0422F4
:0E678900C22BE4F56CF56D75FFDE75FFAD22D9
:1066A500056DE56D7002056C302B14E56B75F064B6
:1066B500A4FFC3E56D9FE56C95F0500375FFA5221A
:0465D9008E418F421E
:1065DD00E4F543F544C3E5449542E5439541501632
:1065ED007FE87E03125FAD7F0112662E0544E54400
:0665FD0070E3054380DF9E
:016603002274
:105F9B0054F0FFE5A054014FF5A0A21292A37F018C
:025FAB007E0076
:045FAD008E658F6608
:105FB100D3E56694FAE5659400500EEFD394004062
:105FC100407E1600DEFD1F80F2856567856668D319
:105FD100E56894FAE567940040157FFA7E00125F48
:105FE100AD74062568F56874FF3567F56780E0D301
:105FF100E5669400E56594004007AF68AE67125FFF
:01600100ADF1
:01600200227B
:10600300754A00754B00754C447B007A0079427DDC
:01601300028A
:086014008B468A4789488D493B
:10601C007F0112662EAB4AAA4BA94C1214CC240059
:10602C00FFE5F034E0FE85464D85474E85484FE44C
:10603C00FDEDC39549501BEF2DF582E43EF583E44D
:10604C0093AB4DAA4EA94F8D827583001214620D2D
:0F605C0080DFAB4AAA4BA94CE48549F002152F0F
:10572800754212754334754A00754B00754C447BBD
:07573800007A0079427D02B6
:08573F008B468A4789488D4919
:105747007889E664F160030257DC126789C2AFE427
:10575700F58443B701758F01AB4AAA4BA94C1214C4
:10576700CC2400FFE5F034E0789AF608EFF6AA4774
:10577700A948789EA64608C6EAC608C6E9C6E478D8
:105787009CF6789CE6C395495032789ECBE6CB08C9
:105797000806E618CAE6CA70010614F912140A7850
:1057A7009DF6E6FF789A0806E618CCE6CC70010667
:1057B70014F5828C83EFF0789C0680C6E4F58F534E
:1057C700B7F0AB4AAA4BA94C8549F012152FD2AFB7
:0557D700E4FF1267026F
:0157DC0022AA
:106438007889E664F17046C2AF126789E4F584434F
:10644800B701758F03789B76E008F6789AF6789B03
:10645800E6FE08E6F5828E83E4F07F0112662E7868
:106468009CE426F618740236F61806E6C39408402B
:0D647800DDE4F58F53B7F0D2AFFF126702DD
:0164850022F4
:10588D00126438E4F544F545F54A754B00754C4402
:10589D00FB7A0079097D1612573F125728E4F5411E
:1058AD00E541C378A1965073E4F540AB76AA77A98C
:1058BD007875F01FE540A4F58285F08312142360FE
:1058CD0056E54075F01FA429F9EA35F0FA90000D60
:1058DD001216C97885E68541F0A429F9EA35F0FA62
:1058ED00EBC0E0EAC0E0E9C0E0AB76AA77A9787535
:1058FD00F01FE540A4F58285F083121423FD754A4F
:10590D0000754B00754C44D0E0F9D0E0FAD0E0FBC7
:10591D0012573F0540809405418085125728E47841
:02592D0089F6F9
:01592F002255
:10566A00E4F544F545F541F54A754B00754C44FBA4
:10567A007A0079097D16126014126003E5436434D6
:10568A007004E54264127003434101E4F540E540C9
:10569A00C378A1965073E4F53FAB76AA77A97875DB
:1056AA00F01FE53FA4F58285F0831214236056E5C6
:1056BA003F75F01FA429F9EA35F0FA90000D121689
:1056CA00C97885E68540F0A429F9EA35F0FAEBC0F5
:1056DA00E0EAC0E0E9C0E0AB76AA77A97875F01FE6
:1056EA00E53FA4F58285F083121423FD754A0075FF
:1056FA004B00754C44D0E0F9D0E0FAD0E0FB1260E0
:10570A0014053F809405408085126003E5436434A4
:0D571A007004E54264127003434102AF4188
:01572700225F
:02618F008F631C
:10619100302C5743A0F075840F75A60FC2A3D2A26D
:1061A100125FA9D2A1E4F5647F0A7E00125FAD30CF
:1061B100A7090564E564C394C840EDC2A1125FA9B3
:1061C100C2A275840F75A6FF125FA9E563125F9BDA
:1061D100D2A1125FA9C2A1125FA9E563C4125F9B9C
:0A61E100D2A1125FA9C2A1125FA9AA
:0161EB002291
:10654F008F4153A00FE54154F042A0D2A1125FA991
:10655F00C2A1125FA953A00FE541C454F042A0D2CB
:10656F00A1125FA9C2A1125FA97F647E00025FAD75
:105F2200E4F53FF540C2A1C2A2C2A375840F75A6D3
:105F3200FF53A00143A020D2A17F01FE125FADC298
:105F4200A17F017E001265D97F2012654F43A0F028
:105F520075840F75A60FC2A3D2A2125FA9D2A17F28
:105F6200647E00125FAD30A703C22C22D22CC21273
:105F72007F2412618FC2127F0912618FC2127F20A9
:105F820012618FC2127F0C12618FC2127F011261E5
:085F92008FC2127F0612618F1D
:015F9A0022E4
:0D67B100C2127F0112618FE4FDFF026754E8
:10675400ED5403C43354E0FEEF541F44804EFFC293
:046764001202618F2D
:106768008F62C3E562648094A04005D21212618FE3
:03677800AF6222EB
:10667E008B798A7A897BAB79AA7AA97B12140A6004
:10668E0015057BE57B7002057A14F912140AFFD208
:07669E001212618F80E0225F
:10497B00202020202020202020200025622A626475
:10498B000025622A62750025622A640025622A7559
:10499B000025622A2E33660025622A6C640025628C
:1049AB002A6C7500253262643A2573002020202082
:1049BB0020202020004E6F207661726961626C6549
:1049CB007320646566696E656400202020202020BA
:1049DB002020202020202020202020202000455394
:1049EB004320454E5445522020202D202020202BA3
:1049FB0020200045534320454E5445522020505211
:104A0B004556204E45585400455343202020202026
:104A1B0020202050524556204E455854005061726C
:104A2B00616D6574657273207772697474656E005D
:104A3B00746F20666C617368206D656D6F72792E73
:104A4B0000F470000000F76E000000FAE4000000B4
:104A5B00FD6D0000000000000000036B000000066D
:104A6B004D00000009470000000C5400000000003E
:104A7B00000000016D0000000267000000037300DE
:104A8B000000046D000000056800000006410000F6
:104A9B0000074B00000008DF43000009DF46000061
:104AAB0014487A000015506100001662610000176F
:104ABB0057000000185600000019F40000001A54AB
:104ACB000000001B6C2F73001C52504D001D460044
:104ADB0000005A250000005B52504D005C636E7461
:104AEB00005D7800000000000000000235000000AF
:104AFB004E6F6465204164720000090000000000E5
:104B0B000000003F8000000000000235000000475D
:104B1B007270204164720000000B00000000000066
:104B2B0000003F8000000000000032000004466CD3
:104B3B00617368000000000000000000000000002E
:104B4B00000000000000000000320000045265620B
:104B5B006F6F7400000000000000000000000000F8
:074B6B000000000000000043
:1060A400C1A3C12AC129C12441035D00011F0444C5
:1060B400035E00000000440355000000004403593F
:0C60C40000000000C125C126C127C12832
:064520008B3E8A3F89403A
:10452600900001121423B4381B85414985424A85FF
:10453600434B754C00754D087B017A037962126214
:10454600F4024762E4900362F0AB3EAA3FA94090B2
:104556000002121423605CE4F544E54475F005A4FA
:10456600244CF582E4344AF583E493FF6015AB3EB0
:10457600AA3FA940900002121423FEEF6E600405C4
:104586004480D7E54475F005A4244CF582E4344A0A
:10459600F583E493601DE54475F005A4244DF97494
:1045A6004A35F07549FFF54A894B7B017A037962F2
:1045B600126246AB3EAA3FA9409000011214236046
:1045C6005CE4F544E54475F005A4247EF582E43404
:1045D6004AF583E493FF6015AB3EAA3FA9409000DD
:1045E60001121423FEEF6E6004054480D7E544757E
:1045F600F005A4247EF582E4344AF583E493601D35
:10460600E54475F005A4247FF9744A35F07549FF31
:10461600F54A894B7B017A0379621262467B017AFD
:1046260003796212000E8F45AB3EAA3FA9401214D1
:104636000A14601D14605E24FE70030246E424041E
:1046460060030247627BFF7A49797B126604024760
:1046560062AB3EAA3FA940900004121423C330E186
:104666001A740A9545F549AB41AA42A94312140AA0
:10467600F54A7BFF7A49798602475F740A9545F5C4
:1046860049AB41AA42A94312140AF54A7BFF7A496B
:10469600798C02475FAB3EAA3FA9409000041214F2
:1046A60023C330E11D740A9545F549AB41AA42A9D9
:1046B600431214CCF54B85F04A7BFF7A4979920276
:1046C600475F740A9545F549AB41AA42A9431214BE
:1046D600CCF54B85F04A7BFF7A497997807BAB3ED8
:1046E600AA3FA94090000412142330E020C3740AA4
:1046F6009545F549AB41AA42A9431215998F4D8EAE
:104706004C8D4B8C4A7BFF7A49799C804CAB3EAAF8
:104716003FA940900004121423C330E11F740A9588
:1047260045F549AB41AA42A9431215998F4D8E4CC6
:104736008D4B8C4A7BFF7A4979A3801D740A954577
:10474600F549AB41AA42A9431215998F4D8E4C8D5E
:104756004B8C4A7BFF7A4979A9123E9F7B017A03EB
:054766007962126604F7
:01476B00222B
:08238500AB3BAA3CA93D7DFF22
:10238D008D418B3E8A3F89409000011214236438A1
:10239D007003022B91AB3EAA3FA94012140A24FEF2
:1023AD0070030225F224FE700302284B2403600300
:1023BD00022B9190000412142320E1030224ACABF4
:1023CD003EAA3FA94090001812162FC000C001C0B0
:1023DD0002C003AC41EC121045D003D002D001D0A5
:1023ED0000120E28C004C005C006C007900351E0BE
:1023FD00FC121045D003D002D001D000120D3712BF
:10240D001079900351EFF0AB3EAA3FA94090001414
:10241D001215B990001012162F120FCE7003022B49
:10242D0091AB3EAA3FA9409000101215B9C004C04F
:10243D0005C006C007900351E0FC121045A804A981
:10244D0005AA06AB07D007D006D005D004120FCED3
:10245D005014AB3EAA3FA9409000101215B91210AE
:10246D0079900351EFF0AB3EAA3FA94090001412B2
:10247D0015B9C004C005C006C007900351E0FC1299
:10248D001045A804A905AA06AB07D007D006D005AC
:10249D00D004120FCE60025003022B910225DDE510
:1024AD0041F4704CAB3EAA3FA9409000101215B9F3
:1024BD00C004C005C006C007900351E0FCE4121033
:1024CD0045A804A905AA06AB07D007D006D005D0AC
:1024DD0004120FCE701AAB3EAA3FA9409000141201
:1024ED0015B990001012162F120FCE6003022B910A
:1024FD00AB3EAA3FA94090001812162FC000C00194
:10250D00C002C003AC41EC121045D003D002D00183
:10251D00D000120E28C004C005C006C0079003519C
:10252D00E0FCE4121045D003D002D001D000120D12
:10253D0037121079900351EFF0AB3EAA3FA94090AE
:10254D0000141215B990001012162F120FCE700331
:10255D00022B91AB3EAA3FA9409000101215B9C0B5
:10256D0004C005C006C007900351E0FCE4121045FD
:10257D00A804A905AA06AB07D007D006D005D0043C
:10258D00120FCE5014AB3EAA3FA940900010121569
:10259D00B9121079900351EFF0AB3EAA3FA94090CC
:1025AD0000141215B9C004C005C006C00790035130
:1025BD00E0FCE4121045A804A905AA06AB07D00754
:1025CD00D006D005D004120FCE60025003022B911D
:1025DD00AB3EAA3FA9409000141215B91210799084
:1025ED000351EFF022AB3EAA3FA940900004121414
:1025FD002320E1030226F090001812162FC000C010
:10260D0001C002C003AC41EC121045D003D002D082
:10261D0001D000120E28C004C005C006C0079003EB
:10262D0051E0FCA3E0FDEC121040D003D002D0012C
:10263D00D000120D37121079900351EEF0A3EFF088
:10264D00AB3EAA3FA9409000141215B9900010128C
:10265D00162F120FCE7003022B91AB3EAA3FA9404D
:10266D009000101215B9C004C005C006C007900334
:10267D0051E0FCA3E0FDEC121040A804A905AA0648
:10268D00AB07D007D006D005D004120FCE5017AB34
:10269D003EAA3FA9409000101215B912107990036F
:1026AD0051EEF0A3EFF0AB3EAA3FA94090001412FB
:1026BD0015B9C004C005C006C007900351E0FCA3C6
:1026CD00E0FDEC121040A804A905AA06AB07D0073F
:1026DD00D006D005D004120FCE60025003022B910C
:1026ED00022833E541F4704FAB3EAA3FA94090005C
:1026FD00101215B9C004C005C006C007900351E003
:10270D00FCA3E0FDE4121040A804A905AA06AB073E
:10271D00D007D006D005D004120FCE701AAB3EAA4A
:10272D003FA9409000141215B990001012162F12E7
:10273D000FCE6003022B91AB3EAA3FA9409000182B
:10274D0012162FC000C001C002C003AC41EC121024
:10275D0045D003D002D001D000120E28C004C00510
:10276D00C006C007900351E0FCA3E0FDE412104049
:10277D00D003D002D001D000120D37121079900382
:10278D0051EEF0A3EFF0AB3EAA3FA940900014121A
:10279D0015B990001012162F120FCE7003022B9147
:1027AD00AB3EAA3FA9409000101215B9C004C00558
:1027BD00C006C007900351E0FCA3E0FDE4121040F9
:1027CD00A804A905AA06AB07D007D006D005D004EA
:1027DD00120FCE5017AB3EAA3FA940900010121514
:1027ED00B9121079900351EEF0A3EFF0AB3EAA3F72
:1027FD00A9409000141215B9C004C005C006C00749
:10280D00900351E0FCA3E0FDE4121040A804A905DB
:10281D00AA06AB07D007D006D005D004120FCE60A4
:10282D00025003022B91AB3EAA3FA9409000141217
:10283D0015B9121079900351EEF0A3EFF022AB3ED3
:10284D00AA3FA94090000412142320E00302290D91
:10285D00900351E0F8A3E0F9A3E0FAA3E0FBC00078
:10286D00C001C002C003AB3EAA3FA94090001812A0
:10287D00162FC000C001C002C003AC41EC121045C0
:10288D00D003D002D001D000120E28D003D002D038
:10289D0001D000120D3790035112166BAB3EAA3FBB
:1028AD00A9409000101215B9900351E0F8A3E0F97A
:1028BD00A3E0FAA3E0FB120FCE5012AB3EAA3FA944
:1028CD00409000101215B990035112166BAB3EAA31
:1028DD003FA9409000141215B9900351E0F8A3E000
:1028ED00F9A3E0FAA3E0FB120FCE60025003022B16
:1028FD0091AB3EAA3FA9409000141215B9022B8B43
:10290D00AB3EAA3FA94090000412142320E103021C
:10291D002A2890001812162FC000C001C002C00353
:10292D00AC41EC121045D003D002D001D000120EF4
:10293D0028C004C005C006C007900351E0FCA3E009
:10294D00FDA3E0FEA3E0FFEC12103BD003D002D0BC
:10295D0001D000120D3712107990035112166BAB86
:10296D003EAA3FA9409000141215B99000101216FE
:10297D002F120FCE7003022B91AB3EAA3FA94090B0
:10298D0000101215B9C004C005C006C00790035150
:10299D00E0FCA3E0FDA3E0FEA3E0FFEC12103BA8DA
:1029AD0004A905AA06AB07D007D006D005D004129E
:1029BD000FCE5015AB3EAA3FA9409000101215B98D
:1029CD0012107990035112166BAB3EAA3FA940909D
:1029DD0000141215B9C004C005C006C007900351FC
:1029ED00E0FCA3E0FDA3E0FEA3E0FFEC12103BA88A
:1029FD0004A905AA06AB07D007D006D005D004124E
:102A0D000FCE60025003022B91AB3EAA3FA940901E
:102A1D0000141215B9121079022B8BE541F4705583
:102A2D00AB3EAA3FA9409000101215B9C004C005D5
:102A3D00C006C007900351E0FCA3E0FDA3E0FEA398
:102A4D00E0FFE412103BA804A905AA06AB07D007C6
:102A5D00D006D005D004120FCE701AAB3EAA3FA9F6
:102A6D00409000141215B990001012162F120FCEAF
:102A7D006003022B91AB3EAA3FA94090001812169D
:102A8D002FC000C001C002C003AC41EC121045D0F4
:102A9D0003D002D001D000120E28C004C005C0061C
:102AAD00C007900351E0FCA3E0FDA3E0FEA3E0FF0F
:102ABD00E412103BD003D002D001D000120D37121A
:102ACD00107990035112166BAB3EAA3FA9409000AE
:102ADD00141215B990001012162F120FCE7003029A
:102AED002B91AB3EAA3FA9409000101215B9C0041E
:102AFD00C005C006C007900351E0FCA3E0FDA3E0B4
:102B0D00FEA3E0FFE412103BA804A905AA06AB073B
:102B1D00D007D006D005D004120FCE5015AB3EAA6B
:102B2D003FA9409000101215B9121079900351125F
:102B3D00166BAB3EAA3FA9409000141215B9C00404
:102B4D00C005C006C007900351E0FCA3E0FDA3E063
:102B5D00FEA3E0FFE412103BA804A905AA06AB07EB
:102B6D00D007D006D005D004120FCE60174015AB9C
:102B7D003EAA3FA9409000141215B9121079900386
:052B8D005112166B223D
:106516008F3EE92405F9E43AFA78627C037D017E30
:10652600007F081213E4E490036AF0853E49754A39
:1065360001754B03754C627BFF7A4979AF123E9F1A
:096546007BFF7A4979B702660473
:10332D00302318126797E47B2C7A01F9F8C3121534
:10333D007540030238DDC2231267B1126797A804E6
:10334D00A905AA06AB0790035EE0FCA3E0FDA3E090
:10335D00FEA3E0240AFFE43EFEE43DFDE43CFCD385
:10336D0012157550030238DD12679790035E121621
:10337D006B202A10C2081238DEEF70030238CDD24E
:10338D002A0238CD302911753BFF753C4A753DF643
:10339D00E51F14789BF6801085763B85773C857804
:1033AD003D787DE614799BF7789BE6FFC394035037
:1033BD0005E408F6801A90035DE0FE7002800EEEC3
:1033CD0090035DB50705E024FE8002E014789CF6BD
:1033DD00787DE67011FDFF1267547BFF7A4979C045
:1033ED00123E9F023508E4789AF6789AE6FDC3946A
:1033FD00034003023508E4FF126754789AE6FF781C
:10340D009CE62FFFE433FE90035DE07C00B50708DA
:10341D00ECB506047F3E80027F20126768789AE63D
:10342D00FD7F01126754789AE6FF789CE62FFFE442
:10343D0033FE18E6FDD3EF9D7480F86E98400C7B3B
:10344D00FF7A4979D5123E9F023502789AE6FF78C8
:10345D009CE62FFFE433FE7C007D1F121484AB3BF2
:10346D00E53D2FF9E53C3EFAC001799CE7789A26B7
:10347D00FFD001126516789AE6FD7F0A1267543067
:10348D002433789AE6FF789CE62FFFE433FE900311
:10349D005DE07C00B5071EECB5061A7D1F12148485
:1034AD00AB3BE53D2FF9E53C3EFA75410175420315
:1034BD00754351803D789AE6FF789CE62FFFE43303
:1034CD00FE7C007D1F121484AB3BE53D2FF9E53CDE
:1034DD003EFAC003C002C001E53D2FF9E53C3EFABE
:1034ED0090000D1216C98B418A428943D001D0023A
:1034FD00D003124520789A060233F790035DE075EC
:10350D00F01FA430290C24F6F9744A35F0753BFFF1
:10351D00800A2578F9E57735F085763BF53C893DD0
:10352D002024030236CF7D03E4FF1267547BFF7A1C
:10353D004979E9126604201705302502C224301896
:10354D005B202658C224AB3BAA3CA93D12140AFFAE
:10355D007E0090000D1216C9A801AC02AD037B01CF
:10356D007A0379511213E430291390035DE0FF6063
:10357D000464017027D21B788976F1801F90035D5A
:10358D00E0FF12476CAB3BAA3CA93D90000412141E
:10359D002330E50890035DE0FF125CA230190F2087
:1035AD00270C12238512679790035512166B30194D
:1035BD002D126797A804A905AA06AB07900355E03D
:1035CD00FCA3E0FDA3E0FEA3E02446FFE43EFEE401
:1035DD003DFDE43CFCD312157540031223853019D3
:1035ED0036126797A804A905AA06AB07900355E004
:1035FD00FCA3E0FDA3E0FEA3E024F4FFEE3401FE06
:10360D00E43DFDE43CFCD3121575400BAB3BAA3CED
:10361D00A93D7DF712238D20190A900355121677B7
:10362D0000000000301A17202814AB3BAA3CA93D1E
:10363D007D0112238D12679790035912166B301A64
:10364D0035126797A804A905AA06AB07900359E0A0
:10365D00FCA3E0FDA3E0FEA3E02446FFE43EFEE470
:10366D003DFDE43CFCD3121575400BAB3BAA3CA9C8
:10367D003D7D0112238D301A36126797A804A905D6
:10368D00AA06AB07900359E0FCA3E0FDA3E0FEA35F
:10369D00E024F4FFEE3401FEE43DFDE43CFCD312E6
:1036AD001575400BAB3BAA3CA93D7D0912238D300E
:1036BD001A030238CD90035912167700000000024C
:1036CD0038CD7D03E4FF126754AB3BAA3CA93D9076
:1036DD0000181215B9E4FBFAF9F8120FCE400FAB32
:1036ED003BAA3CA93D90000412142330E2087BFF55
:1036FD007A4979FE80067BFF7A4A79131266042097
:10370D001716302513302909C229E490035DF08086
:10371D0007C22AD2081238DE2018030237BC302621
:10372D00030237BCAB3BAA3CA93D12140AFFD3944C
:10373D00045032EF9400402D9000181215B9E4FB9F
:10374D00FAF9F8120FCE501DD224AB3BAA3CA93D7D
:10375D0012140AFF7E0090000D1216C978517C03D9
:10376D007D011213E430293790035DE06402702F60
:10377D00D21B788976F11267B1E4FDFF1267547B95
:10378D00FF7A4A79281266047D01E4FF1267547BA3
:10379D00FF7A4A793B1266047FB87E0B1265D930E9
:1037AD00290D90035DE0B40306E4F58475EF103048
:1037BD00192B20272890035DE07013202907787DB1
:1037CD00E614F0800FE51F1490035DF08006900362
:1037DD005DE014F012679790035512166B3019497E
:1037ED00126797A804A905AA06AB07900355E0FC3C
:1037FD00A3E0FDA3E0FEA3E02446FFE43EFEE43D8E
:10380D00FDE43CFCD3121575401F90035DE0701371
:10381D00202907787DE614F0800FE51F1490035DD5
:10382D00F0800690035DE014F020190A9003551204
:10383D00167700000000302906789AA61F800678BA
:10384D007DE6789AF6301A1D20281A90035DE00463
:10385D00FF789AE6FEEF8EF084E5F0F01267979010
:10386D00035912166B301A3B126797A804A905AAC3
:10387D0006AB07900359E0FCA3E0FDA3E0FEA3E037
:10388D002446FFE43EFEE43DFDE43CFCD3121575F9
:10389D00401190035DE004FF789AE6FEEF8EF08410
:1038AD00E5F0F0201A0A9003591216770000000077
:1038BD0030190D301A0A202907E490035DF0D22942
:1038CD00A2179225A2189226A2199227A21A92281F
:0138DD0022C8
:100D30000210E5E86480F8E933E83360110460F0FC
:100D4000ED33EC337009E8FCE9FDEAFEEBFF220429
:100D500060DED3EB9FEA9EE99DE8C2E78CF0C2F724
:100D600095F0400CE8CCF8E9CDF9EACEFAEBCFFBF0
:100D70001210B085D0F05804700320D5B3E8047089
:100D8000075002B2D50210EF92D5EC0460F7E4CC24
:100D9000C0E0C398F8603B94186008400DD0E0FBB9
:100DA0000210C7E4FBFAC9FC8028E830E406E4C975
:100DB000FBE4CAFCE830E305E4C9CACBFCE854070D
:100DC0006010F8C3E913F9EA13FAEB13FBEC13FC18
:100DD000D8F130F52FC3E49CFCEF9BFFEE9AFEEDBB
:100DE00099FDD0E0FBEF4E4D4C701222DB03021058
:100DF000ECEC2CFCEF33FFEE33FEED33FDED30E792
:100E0000EB0210C7EF2BFFEE3AFEED39FDD0E0FB11
:100E100050130BBB00030210EFED13FDEE13FEEFBA
:080E200013FFEC13FC0210C7E4
:100E2800EC4D6011E8497017ED33EC3304600DE4C4
:100E3800FCFFFEFD22E933E8330470F80210E512E6
:100E480010B058046009E4CC2481500628500902E7
:100E580010EF2840030210ECC0E0EB4A7044B98060
:100E680006D0E0FB0210DBEF4E701CBD8008EBFFE4
:100E7800EAFEE9FD80EBE98DF0A4FEE5F0020F1132
:100E8800E9CDF9EAFEEBFFEF89F0A4FCE5F0CE89A5
:100E9800F0A42EFFE435F0CD89F0A42DFEE435F062
:100EA8008067EF4E7005BD80D780C3EF8BF0A4AC90
:100EB800F0EE8BF0A42CFCE435F0F8EF8AF0A42CCB
:100EC800E5F038FCE433CB8DF0A42CFCE5F03BF8DE
:100ED800EE8AF0A42CFCE5F038F8E433CF89F0A4CE
:100EE8002CFCE5F038CF3400CE89F0A42FFFE5F0D4
:100EF8003EFEE433C98DF0A42EFEE5F039CD8AF02C
:100F0800A42FFFE5F03EFEE43DFD33D0E0FB5007A3
:100F18000BBB000F0210EFEC2CFCEF33FFEE33FE9F
:060F2800ED33FD0210C7CD
:100F2E000210EFEC5D046005E8590470030210E551
:100F3E001210B0580460F6EC4860F2EC7004FDFE3E
:100F4E00FF22C860DB2481C85009C3986002500696
:100F5E000210EC9850CAF582E9294B4A7005AB8213
:100F6E000210DB75F0007C1A7880C3EF9BEE9AEDD1
:100F7E0099400DC3EF9BFFEE9AFEED99FDE842F00E
:100F8E00DC23ACF0D0E0FFD0E0FED0E0FDAB822061
:100F9E00E7101BEB60BAEC2CFCEF33FFEE33FEEDEB
:100FAE0033FD0210C7E803F830E705C0F075F00016
:100FBE00EF2FFFEE33FEED33FD40B830E7C280AACF
:100FCE0074F8CC6480CCC86480C8F582046043C3D6
:100FDE00EB9FF5F0EA9E42F0E99D42F0E89C45F069
:100FEE0060305018E5825FFFE582F42B5582FB508E
:100FFE00210ABA001D09B90019088016E5825BFBAB
:10100E00E582F42F5582FF50090EBE00050DBD007E
:10101E00010CC3EB9FF5F0EA9E42F0E99D42F0E829
:0D102E009C45F06007CC4820E701B3EC22A0
:10103B0075F020800E75F010800575F0087D007E30
:10104B00007F003392D530D503121567EC33401077
:10105B00EF33FFEE33FEED33FDEC33FCD5F0ED2239
:0E106B00E5F0247EA2D513CC92E7CDCEFF2275
:10107900EDD2E7CD33EC3392D524814006E4FFFE6F
:10108900FDFC22FCE4CFCECDCC24E0501174FF80CE
:10109900EDC3CC13CCCD13CDCE13CECF13CF04706B
:0710A900F030D5DE021567EF
:103E3D00E55D2449F8E6055D2278463010027849A3
:103E4D00E475F0011216B902140A2009EB7F2ED287
:103E5D00098018EF540F2490D43440D4FF300D0B4B
:103E6D00EF24BFB41A0050032461FFE55E60021514
:103E7D005E0561E5617002056030100D7846E475F0
:103E8D00F0011216B9EF0214500267687403D210D4
:103E9D008003E4C210F55D8B468A478948E4F55EE0
:103EAD00F560F561E55E60077F20123E7880F5755F
:103EBD005FFFC20AC209C20BC20CC20EC20FC211F1
:103ECD00123E46FF700D3010057F00123E89AF6126
:103EDD00AE6022B4255FC2D5C20D123E46FF24D07E
:103EED00B40A00501A75F00A785E30D50508B6FF91
:103EFD000106C6A426F620D5047002D20C80D92462
:103F0D00CFB41A00EF5004C2E5D20D024176D20AA9
:103F1D0080C6D20980C0D20B80BCD2D580BAD20E59
:103F2D0080B47F20123E78200B077401B55E0040EF
:103F3D00F1123E3DFF123E78023EB1D211D20F80FA
:103F4D0095123E3DFB123E3DFA123E3DF94A4B7035
:103F5D0006796D7A427BFF200B2EE55E602A7E008E
:103F6D008E8275830012142360060EEE655F70F06D
:103F7D00C2D5EBC0E0EAC0E0E9C0E0EE1241D6D018
:103F8D00E0F9D0E0FAD0E0FB12140AFF60AAEBC012
:103F9D00E0EAC0E0E9C0E0123E78D0E02401F9D0BB
:103FAD00E03400FAD0E0FBE55F0460DCD55FD9803A
:103FBD0087D20B80A21241B960F7E55F7001041240
:103FCD001125A95F600DE55F600914F55F12426070
:103FDD00EF60F3EA30E702F404C3995077EAF42571
:103FED005F0430E701E404F55F800D1241B960C153
:103FFD00EA055F255F121125EA785CF630E701E4EA
:10400D00255F04D55F04200E01141241D6E4C0E0F3
:10401D00124260785CE6601320E70714F6123E60EA
:10402D00802204F6D0E014C0E07F00123E60E55F10
:10403D006007123E57155F800B300E03123E57D0AE
:10404D00E0023EB1D0E00480C51241B960A0E55F49
:10405D0004121125785CEAF6E55F200E026001047A
:05406D0024041241D6FD
:1040720074FF04C0E0124260123E60E55F200E024F
:104082006003123E57D0E0B55FE87F45123E6A7882
:104092005CE67F2B30E7047F2DF404C0E0123E780B
:1040A200D0E075F00A84C0F0123E61D0E0123E61A9
:1040B200023EB1791080027908C20FC2118008D283
:1040C200D5790A8004790AC2D5E55F047002F55FEA
:1040D200E4FAFDFEFF123E3DFC7B08200A13123E6D
:1040E2003DFD7B1030090A123E3DFE123E3DFF7B34
:1040F20020EC3382D592D55013C3E43009069FFFDA
:10410200E49EFEE4200A039DFDE49CFCE4CBF8C29D
:104112000AEC700CCFCECDCCE824F8F870F38017FF
:10412200C3EF33FFEE33FEED33FDEC33FCEB33FB39
:10413200994002FB0FD8E9EB300A05F8D0E0C448F9
:10414200B20AC0E00AEC4D4E4F78207B0070C2EA02
:10415200B55F0040BCC0E01241D8D0F0D0E0200AE8
:1041620004C4C0E0C4B20AC0F0123E61D0F0D5F07F
:10417200EB023EB11216F93F4E5340B5583F1F4C69
:104182003F1B4240B94F40C14440C1493F344340C4
:10419200C7553FF8464056453FC247428D503F23E0
:1041A2002D3F272E3F4A2B3F2B233F482042762A82
:1041B2003EE34800003F42E55FB4FF03755F06122D
:1041C2003E3DFC123E3DFD123E3DFE123E3DFF785D
:1041D20055021154790AA2D5200C14300E09B910D7
:1041E200020404B9080104A2D5200F0250010420E0
:1041F2000B68920BB55E005034C0E07F20300C1982
:104202007F30A20B720F720E500F12422FC20BC2DE
:104212000FC20EC2117F30800F300E03E9C0E012D0
:104222003E78300E03D0E0F9D0E0B55ECC300E1708
:104232007F30B9100C123E787F58300D077F78809E
:1042420003B90803123E78300B057F2D023E787FBA
:10425200202011F87F2B200FF322920B80CF7F00BA
:10426200B4070050052455F8E6FF22286E756C6CE1
:104272002900D20A123E3D300AF8C20A785E30D5D1
:104282000108F6023EE32D50434958123E3D2403F5
:10429200B405004001E490428893123E69743A12D8
:0A42A2003E69D20C755E040240B5BF
:1057DD008F478E468D458C4474FFFFFEFDFCAB4715
:1057ED00AA46A945A844C3121575602C7F807E96E4
:1057FD007D187C4BAB47AA46A945A844120FCE6035
:10580D000250157F807E967D187CCBAB47AA46A9AA
:10581D0045A844120FCE5009AF47AE46AD45AC4436
:10582D0022AF47AE46AD45AC441210798F4B8E4A30
:10583D008D498C48EC12103BC8ECC8C9EDC9CAEEB5
:10584D00CACBEFCBAF47AE46AD45AC44120D33E4FA
:10585D00FBFAF9F8120FCE601A401874FF254BF5BC
:10586D004BE54A34FFF54AE54934FFF549E548343F
:10587D00FFF548AF4BAE4AAD49AC48EC12103B2298
:105269008F3E8E3D8D3C8C3BE4FFFE7D807C3FABC9
:105279003EAA3DA93CA83B120FCE7009AF3EAE3DF8
:10528900AD3CAC3B22AF3EAE3DAD3CAC3B1210FA5F
:10529900FBAF42AE41AD40AC3F1210FAFFBF01086F
:1052A900E4FFFE7D807C3F22EF64046022EB64040E
:1052B900601DBB0127E4FFFEFDFCAB42AA41A940EA
:1052C900A83F120FCE60084006E4FFFEFDFC2274E1
:1052D900FFF542F541F540F53F025377E4F543F513
:1052E90044FFFEFDFCAB3EAA3DA93CA83B120FCEF4
:1052F900504BAF42AE41AD40AC3F1210798E438F57
:1053090044AC43AD44EC121040C8ECC8C9EDC9CA5D
:10531900EECACBEFCBAF42AE41AD40AC3F120D333D
:10532900E4FBFAF9F8120FCE70A5AF3EAE3DAD3CE5
:10533900AC3B1211148F3E8E3D8D3C8C3BAF3EAE83
:105349003DAD3CAC3B12503DAB42AA41A940A83F00
:10535900120E28125A048F428E418D408C3FE5442B
:1053690030E00B1211148F428E418D408C3FAF42B9
:07537900AE41AD40AC3F2244
:1010B000E9D2E7C933E833F892D5EDD2E7CD33EC86
:0710C00033FC5002B2D522FF
:1010C700EC30E7100FBF000C0EBE00080DBD00048A
:1010D7000BEB6014A2D5EB13FCED92E7FD2274FF36
:1010E700FCFDFEFF22E480F8A2D574FF13FC7D808F
:0310F700E480EFA3
:1010FA00ED33EC33601004700FED547F7005740209
:0A110A0092E2227404220422E4227F
:10111400ED33EC33600A047003BD8004ECB2E7FCE9
:0111240022A8
:10112500F920E72824F950037907E4F42402FB1891
:10113500DBFDE624FB5014E9600DE4F618E604F641
:0F114500B40A08E4F6D9F57401F60A22C2D522DD
:10115400ED33EC3392D5FA602AB4FF33EDC2E77B6A
:10116400FF60067A117979E4227A11798220D50414
:101174007A11797D224E614E002B494E46002D494D
:101184004E4600E47A08F608DAFC7B00740722E88D
:10119400C0E0ECC0E0EDC0E0EEC0E0EFC0E0EA7516
:1011A400F010A4CAABF075F04DA42BFBE435F0FCB1
:1011B400EA2410FAEB34C5FBEC34D9FCEDC2E7FFAA
:1011C40075F056A4F42411C5F0F434C58FF0A42AA4
:1011D400E5F03BE43CF620E714121287D0E0FFD0A0
:1011E400E0FED0E0FDD0E0FC120F318014F40412D4
:1011F4001287D0E0FFD0E0FED0E0FDD0E0FC120E7C
:1012040028D0E0F8E6FAEDD2E7CD33EC332482FBC4
:10121400E4C3CF33CFCE33CECD33CD33DBF37B0733
:1012240075F00A846004F6081B0AE5F0F6088FF0EE
:10123400740AA4FFACF08EF0740AA42CFEACF05037
:10124400010C8DF0740AA42CFDE435F0F608DBDE05
:03125400740722FA
:1059CC0033DA929E35B16011377FE5FE3921848937
:1059DC003AAEC3FF3C1D955B3D6358473E75FDF0E9
:1059EC003F3172183F800000C2D50210EF0210E563
:1059FC00BD80FA50F30210ECED33EC330460F17B14
:105A0C003B7AAA79B8783F120E28ED33EC3392D555
:105A1C00247B5011A2D570DB500BED448024045034
:105A2C0004A2D580CEEFFBEEFAEDF9ECF81210796A
:105A3C00EFF582F404FC121045120D37C082905918
:105A4C00CC74091212D6ED33CC33D0F092D525F0AC
:0A5A5C00A2D57001C313CC13FD2284
:105009003E9248DA3ECCCCCD3F2AAAAB4000000004
:105019003F8000003F9837F03FB504F33FD744FC89
:105029003E3172173EB172173F0515913EDE5BD9CD
:10503900D2088002C208EDD2E7F8CD33EC33047010
:105049000BBD800592D50210EF0210E540FBD31489
:1050590060F2F5F07C3FEE7A00C39496C8948B40D9
:10506900230AC89469C8941A401A0AC89468C8944B
:105079001F40110AC8945AC89425400805F07A00BF
:10508900CDC2E7CDC0F08C458D468E478F48EA23C7
:1050990023C0E02419F582E43450F58312161F1257
:1050A9000D37ECC0E0EDC0E0EEC0E0EFC0E0121655
:1050B9000FA845A946AA47AB48120D33D0E0FBD04B
:1050C900E0FAD0E0F9D0E0B2E7F8120F318C458D63
:1050D900468E478F4890500974031212C7A845A9F4
:1050E90046AA47AB48120E28D0E0600F2425F58266
:1050F900E43450F58312161F120D378C458D468EF8
:10510900478F48D0E0C3947FFDE49400FC1210401F
:105119007B187A727931783F120E28A845A946AAD8
:1051290047AB48120D3730080B7BD97A5B79DE78AB
:055139003E120E2822C9
:101257003F8000004120000042C80000447A00009F
:10126700461C400047C35000497424004B18968021
:101277004CBEBC205A0E1BCA6753C21C749DC5AE18
:10128700FB60065407601C23231212B5EB54386029
:10129700091212A11212B0120E28ECF8EDF9EEFAAB
:1012A700EFCB22EB1212B080F1543803241C9012BA
:1012B70057FE93FC0EEE93FD0EEE930ECE93FF2298
:1012C700C0E0EFFBEEFAEDF9ECF8120E28D0E0F5EE
:1012D700F0EFFBEEFAEDF9ECF812160FA3A3A3A3B8
:1012E700E8C0E0E9C0E0EAC0E0EBC0E0C0F0120E01
:1012F7002812161FA3A3A3A3120D37D0F0D0E0FB2B
:0D130700D0E0FAD0E0F9D0E0F8D5F0D42223
:03000000025C1689
:0C5C1600787FE4F6D8FD7581A1025C5D8A
:10131400E709F608DFFA8046E709F208DFFA803EBB
:1013240088828C83E709F0A3DFFA8032E309F608A8
:10133400DFFA8078E309F208DFFA807088828C8310
:10134400E309F0A3DFFA806489828A83E0A3F608C4
:10135400DFFA805889828A83E0A3F208DFFA804C9E
:1013640080D280FA80C680D4806980F28033801075
:1013740080A680EA809A80A880DA80E280CA8033DE
:1013840089828A83ECFAE493A3C8C582C8CCC58356
:10139400CCF0A3C8C582C8CCC583CCDFE9DEE78026
:1013A4000D89828A83E493A3F608DFF9ECFAA9F0A5
:1013B400EDFB2289828A83ECFAE0A3C8C582C8CCFB
:1013C400C583CCF0A3C8C582C8CCC583CCDFEADE14
:1013D400E880DB89828A83E493A3F208DFF980CC76
:1013E40088F0EF60010E4E60C388F0ED2402B4046F
:1013F4000050B9F582EB2402B4040050AF23234516
:06140400822390136473C3
:10140A00BB010689828A83E0225002E722BBFE02E0
:09141A00E32289828A83E4932213
:10142300BB010CE58229F582E5833AF583E022507E
:1014330006E92582F8E622BBFE06E92582F8E222C8
:0D144300E58229F582E5833AF583E49322E2
:10145000BB010689828A83F0225002F722BBFE017B
:02146000F32275
:10146200F8BB010DE58229F582E5833AF583E8F0C0
:10147200225006E92582C8F622BBFE05E92582C86C
:02148200F22254
:10148400EF8DF0A4A8F0CF8CF0A428CE8DF0A42E7C
:02149400FE2236
:10149600C2D5EC30E709B2D5E4C39DFDE49CFCEE71
:1014A60030E715B2D5E4C39FFFE49EFE121834C39D
:1014B600E49DFDE49CFC800312183430D507C3E498
:0614C6009FFFE49EFE22E0
:1014CC00BB010A89828A83E0F5F0A3E022500687EB
:1014DC00F009E71922BBFE07E3F5F009E3192289AD
:0B14EC00828A83E493F5F074019322E0
:1014F700BB0110E58229F582E5833AF583E0F5F033
:10150700A3E0225009E92582F886F008E622BBFE0F
:101517000AE92582F8E2F5F008E222E5832AF58355
:08152700E993F5F0A3E993221A
:10152F00BB010789828A83021889500B09C5F027EE
:10153F00F7C5F01937F722BBFE0D09F8E325F0F3D5
:10154F00C5F019E338F322F889828A837401932551
:08155F00F0C5F0F8E493382216
:0E156700C3E49FFFE49EFEE49DFDE49CFC2295
:10157500EB9FF5F0EA9E42F0E99D42F0E89C45F0CC
:011585002243
:10158600E8600FECC313FCED13FDEE13FEEF13FF43
:03159600D8F12267
:10159900BB010789828A8302189F5005E9F8021660
:1015A90003BBFE05E9F80218AB89828A8302160F8C
:1015B900BB010DE58229F582E5833AF58302189F7F
:1015C9005007E92582F8021603BBFE07E92582F8D0
:1015D9000218ABE58229F582E5833AF58302160FF5
:1015E900BB010789828A8302166B5005E9F8021646
:0A15F9005FBBFE05E9F80218DD22D1
:0C160300E6FC08E6FD08E6FE08E6FF2213
:10160F00E493FC740193FD740293FE740393FF2221
:10161F00E493F8740193F9740293FA740393FB2221
:10162F00BB010DE58229F582E5833AF5830218C4E3
:10163F005007E92582F80218B7BBFE07E92582F8A3
:10164F000218D0E58229F582E5833AF58302161F49
:0C165F00ECF608EDF608EEF608EFF622B7
:0C166B00ECF0A3EDF0A3EEF0A3EFF022F2
:10167700A8828583F0D083D08212168E12168E121E
:10168700168E12168EE473E493A3C583C5F0C58343
:10169700C8C582C8F0A3C583C5F0C583C8C582C8BD
:0116A7002220
:1016A800F5F0C582A4C582C5F0C583A42583F5835A
:0116B800220F
:1016B900FAE6FB0808E6F925F0F618E6CA3AF62232
:1016C900BB010DE58229F582E5833AF5830218F21B
:1016D9005007E92582F80218E9BBFE07E92582F8D7
:1016E9000218FBE58229F582E5833AF5830219049C
:1016F900D083D082F8E4937012740193700DA3A380
:1017090093F8740193F5828883E473740293686093
:06171900EFA3A3A380DF93
:1066040012140A601CFF09E970010AC0E0EAC0E044
:10661400EBC0E0126768D0E0FBD0E0FAD0E0F9808C
:0A662400DF7F0A126768E4FEFF2220
:106246008B468A4789488B4C8A4D894EAB46054812
:10625600E548AA477002054714F912140A70ED744E
:10626600FF2548F54874FF3547F547AB49054BE52B
:106276004BAA4A7002054A14F912140AFFAB4605E6
:1062860048E548AA477002054714F9EF1214507002
:08629600DAAB4CAA4DA94E221F
:10171F00E709F60870FA8046E709F20870FA803E8A
:10172F0088828C83E709F0A370FA807EE309F608BC
:10173F0070FA8076E309F20870FA806E88828C83E3
:10174F00E309F0A370FA806289828A83E0A3F60826
:10175F0070FA805689828A83E0A3F20870FA804A71
:10176F0080D280FA80C680D4806580F2803180106C
:10177F0080A680EA809A80A880DA80E280CA8031D1
:10178F0089828A83ECFAE493A3C8C582C8CCC58347
:10179F00CCF0A3C8C582C8CCC583CC70E9800D89B5
:1017AF00828A83E493A3F60870F9ECFAA9F0EDFBB3
:1017BF002289828A83ECFAE0A3C8C582C8CCC5838C
:1017CF00CCF0A3C8C582C8CCC583CC70EA80DD89B4
:1017DF00828A83E493A3F20870F980CE88F0ED2417
:1017EF0002B4040050C4F582EB2402B4040050BAD2
:0917FF00232345822390176F7328
:1062F4008B468A478948E4F54EF54FE54D154DAE7A
:106304004C7002154C4E6033AB49AA4AA94B121487
:106314000AFFAB46AA47A948054FE54FAC4E7002A9
:10632400054E14F5828C83EF121462EF60CD740174
:10633400254BF54BE4354AF54A80C0AB46AA47A93C
:026344004822ED
:10000E00E4FFFE12140A600C0FEF70010E09E97086
:05001E00F20A80EF2250
:10672000E94A4B70012212140AFF6D700122EF70CA
:0C67300004FBFAF92209E970ED0A80EA86
:10180800EF4E6012EF60010EEDBB010B89828A83F7
:10181800F0A3DFFCDEFA2289F05007F709DFFCA904
:0C182800F022BBFEFCF309DFFCA9F0225B
:105C220002677BE493A3F8E493A34003F68001F2B6
:105C320008DFF48029E493A3F85407240CC8C33383
:105C4200C4540F4420C8834004F456800146F6DF52
:105C5200E4800B010204081020408090606BE47E17
:105C6200019360BCA3FF543F30E509541FFEE49347
:105C7200A360010ECF54C025E060A840B8E493A30E
:105C8200FAE493A3F8E493A3C8C582C8CAC583CA39
:105C9200F0A3C8C582C8CAC583CADFE9DEE780BEF1
:0160D00000CF
:10183400BC000BBE0029EF8DF084FFADF022E4CC98
:10184400F875F008EF2FFFEE33FEEC33FCEE9DEC61
:10185400984005FCEE9DFE0FD5F0E9E4CEFD22EDA7
:10186400F8F5F0EE8420D21CFEADF075F008EF2FF1
:10187400FFED33FD4007985006D5F0F222C398FDE2
:051884000FD5F0EA227F
:10188900C5F0F8A3E028F0C5F0F8E58215827002EA
:061899001583E038F02287
:0C189F00E0FCA3E0FDA3E0FEA3E0FF22BC
:0C18AB00E2FC08E2FD08E2FE08E2FF2279
:0D18B700E6FB08E6F908E6FA08E6CBF822A1
:0C18C400E0F8A3E0F9A3E0FAA3E0FB22A7
:0D18D000E2FB08E2F908E2FA08E2CBF82298
:0C18DD00ECF208EDF208EEF208EFF22247
:0918E900E6FB08E6FA08E6F92224
:0918F200E0FBA3E0FAA3E0F922F7
:0918FB00E2FB08E2FA08E2F9221E
:0C190400E493FB740193FA740293F9223F
:00000001FF
